:10000000002000206D01000099010000990100000E
:100010009901000099010000990100009901000078
:100020009901000099010000990100009901000068
:100030009901000099010000990100009901000058
:100040009901000021A40000ED8700009901000043
:100050006D800000990100002DA40000398A000085
:100060009901000099010000990100008D5A0000DB
:10007000D1120000990100009901000099010000CF
:100080009901000099010000990100009901000008
:100090009901000010B5064C2378002B07D1054BC1
:1000A000002B02D0044800E000BF0123237010BDE4
:1000B0009804002000000000A8BE000008B5084B0E
:1000C000002B03D00748084900E000BF0748036839
:1000D000002B00D108BD064B002BFBD09847F9E759
:1000E00000000000A8BE00009C0400209404002032
:1000F00000000000164B002B00D1144B9D464022FF
:1001000092029A1A924600218B460F461348144ACF
:10011000121A0AF0E0FD0F4B002B00D098470E4B4F
:10012000002B00D098470020002104000D000D484E
:10013000002802D00C4800E000BF0AF09DFD20001E
:1001400029000AF035F80AF081FDC04600000800D9
:1001500000200020000000000000000098040020A3
:10016000A00F0020000000000000000006488047AB
:100170000649074A074B9B1A03DD043BC858D05079
:10018000FBDCFFF7B7FF0000E5020000B4BE000093
:100190000000002098040020FEE7C04680B582B031
:1001A00000AF00F01FF8031C7B60084B5B680F2258
:1001B00013401A1C7B68D3407B60054B7A681A6039
:1001C0007B68181CBD4602B080BDC04600800C4054
:1001D000840F002080B500AF014B181CBD4680BDC8
:1001E00000366E0180B582B000AF344BDB6A344A12
:1001F000134080225201934215D080225201934233
:1002000004D880221201934211D017E0802292017B
:10021000934204D08022D20493420CD00EE0294BAA
:100220001B687B6039E080231B027B6035E0264B36
:100230001B687B6031E0254B7B602EE01F4BDA684A
:10024000E023DB00134080229200934218D08022EA
:100250009200934206D8002B18D08022520093427D
:1002600011D016E0C0229200934206D08022D20024
:1002700093420ED1164B7B600EE0164B7B600BE079
:10028000154B7B6008E0154B7B6005E0144B7B60F1
:1002900002E000237B60C046C046084B1A68E0239A
:1002A0005B0213409B0B01337868191C0AF0FAF8C3
:1002B000031C181CBD4602B080BDC04600800C4027
:1002C000003C0004040000200000002000366E0105
:1002D000406F4001809FD500C0D8A70040B56400A2
:1002E000804F120080B500AFBD4680BD80B500AF25
:1002F00080231B02181CBD4680BDC04680B500AFE0
:10030000FA239B00181CBD4680BDC04680B500AFD7
:10031000024B1B68181CBD4680BDC046040000206F
:1003200080B582B000AF114B7B60114B1B7801226E
:100330005340DBB2002B14D00D4B01221A700CE09D
:100340007B681B689847031C3B603B68002B01D00F
:100350003B6807E07B6804337B607B681B68002B8D
:10036000EED10023181CBD4602B080BD080000205D
:10037000E004002080B584B000AF78603960114B94
:100380001B7801225340DBB2002B02D00E4BFB60E6
:1003900012E07B68002B0DDC7B682C225A430B4B50
:1003A000D3183A68101C191C2C220AF08BFC00236D
:1003B000FB6001E0064BFB60FB68181CBD4604B007
:1003C00080BDC046E004002005001180B404002078
:1003D0000200118080B584B000AF7860134B1B78A9
:1003E00001225340DBB2002B02D0114BFB6017E01F
:1003F000104B1B68002B11DC0E4B1B68591C0D4A5F
:1004000011602C225A430C4BD2187B68101C191C0B
:100410002C220AF057FC0023FB6001E0074BFB6035
:10042000FB68181CBD4604B080BDC046E004002037
:1004300005001180E4040020B404002001001180B4
:1004400080B58CB000AF00F051FA00F0EBF900F08D
:1004500069FA04200C210022002300F075FA042020
:100460000A210022002300F06FFA00200A21002256
:10047000002300F069FA002008210022002300F088
:1004800063FA052003210022002300F05DFA052015
:100490000321402200F0A6FA031CFB62FB6A002B3A
:1004A00001D0FB6A35E03B1C1C4A1A603B1C012250
:1004B0001A743B1C00225A743B1C80225A603B1C5D
:1004C0008022DA603B1C5A683B1C9A603B1C144A31
:1004D0005A613B1C134A9A613B1C134ADA613B1C6C
:1004E000124A1A623B1C124A5A623B1C114A9A6217
:1004F0003B1C181CFFF76EFF031CFB62FB6A002B02
:1005000006D13B1C181C012100F026F800F03EF833
:10051000FB6A181CBD460CB080BDC04650B500003B
:1005200059050000D90500004D060000A90600008D
:10053000650600003905000080B584B000AF786022
:100540000023FB6000F0D2F900F06CF9FB68181C86
:10055000BD4604B080BDC04680B582B000AF7860B3
:100560000A1CFB1C1A70FB1C1B78002B04D00020FB
:10057000082100F00FFA03E00020082100F01EFA25
:100580000023181CBD4602B080BDC04680B582B0B5
:1005900000AF00200A2100F0FDF9062000F0B2F9BA
:1005A0000C4B1B7804221343DBB29AB2BB1D1A809A
:1005B000BB1D181C022100F05FF9022000F0A2F917
:1005C00000200A2100F0FAF90023181CBD4602B0F1
:1005D00080BDC046E804002080B586B000AFF8605A
:1005E000B9607A603B60BB68DB087A6853437B6123
:1005F000BB68802B01D0114B1CE0114B1A687B6942
:10060000D218104B9A4204D93B6800221A600E4B54
:1006100010E00B4B1A683B681A60094B1A687B693B
:1006200059087B6901200340CB185B00D218044BAA
:100630001A600023181CBD4606B080BD0200118060
:10064000100000202C0E00200100118080B582B027
:1006500000AF78603960024B181CBD4602B080BD07
:100660000400118080B586B000AFF860B9607A6090
:100670003B60BB687B6100233B610BE07B69181C1E
:10068000002110220AF027FB7B6910337B613B6954
:1006900001333B613A693B689A42EFD30023181C4F
:1006A000BD4606B080BDC04680B588B000AFF860DA
:1006B000B9607A603B60BB68BB61BB6A0133BB62F7
:1006C00000200A2100F066F9062000F01BF9BB6A41
:1006D0009BB21B029BB2012213439AB21623FB1852
:1006E0001A801623FB18181C022100F0C5F80023FD
:1006F000FB612BE0BB69181C102100F0BDF8BB6941
:100700001033BB61FB6A5A1EFB699A4205D116235E
:10071000FB18012252421A800FE0BB6A9AB2FB69B1
:100720009BB2D3189BB201339BB21B029BB2FF2238
:1007300013439AB21623FB181A801623FB18181CB1
:10074000022100F099F8FB690133FB61FA69FB6A49
:100750009A42CFD3022000F0D5F800200A2100F001
:100760002DF90023181CBD4608B080BD80B582B0AD
:1007700000AF021C3960FB1D1A70FB1D1B78002B9B
:100780000DD0FB1D1B78012B09D0FB1D1B78022B04
:1007900005D0FB1D1B78032B01D0FB1D1B780949DD
:1007A000FB1D1A783B6801209840031C181C131C81
:1007B000DB009B189B00CB1810335860BD4602B07D
:1007C00080BDC0460060004080B582B000AF021C12
:1007D0003960FB1D1A70FB1D1B78002B0DD0FB1D13
:1007E0001B78012B09D0FB1D1B78022B05D0FB1DAC
:1007F0001B78032B01D0FB1D1B780949FB1D1A78C0
:100800003B6801209840031C181C131CDB009B183C
:100810009B00CB1810331860BD4602B080BDC046A7
:100820000060004090B589B000AF0023FB613B1D24
:100830000D4A13CA13C313CA13C30C4B181C01214E
:1008400002F0E8FC3B1D0A4A9A600A4A3B1D101C54
:10085000191C04F009FB074B0A225A65FB69181C96
:10086000BD4609B090BDC04668B500000032040026
:10087000E067350000C0004080B584B000AF78600C
:1008800039600023FB6021E03B68012B03D07B68CB
:10089000012213400DD07B681B78134A101C191CD1
:1008A00004F092FB3B68013B3B607B6801337B605B
:1008B0000CE07B681B880C4A101C191C04F098FB88
:1008C0003B68023B3B607B6802337B603B68002BEC
:1008D000DAD1C046044B1B6920221340FAD0FB68D2
:1008E000181CBD4604B080BD00C0004080B582B079
:1008F00000AF00237B6000F089FF7B68181CBD46B9
:1009000002B080BD80B584B000AF78600023FB608A
:100910007B68181C01F078F8FB68181CBD4604B011
:1009200080BDC04680B582B000AF00237B60054B20
:10093000181C012102F06EFC7B68181CBD4602B039
:1009400080BDC0460082040080B586B000AFF8606C
:10095000B9603B60FB1D1A7000237B61FB1D1B7897
:10096000002B0FD11323FB1804221A70C046FB681A
:10097000D8B2B9681323FB181A783B6803F056FA0B
:100980007B6900E0024B181CBD4606B080BDC04626
:100990000100138080B584B000AF78603960002317
:1009A000FB607B68DAB23B68101C191CFFF70CFF78
:1009B000FB68181CBD4604B080BDC04680B584B03D
:1009C00000AF786039600023FB607B68DAB23B6877
:1009D000101C191CFFF7CAFEFB68181CBD4604B0AA
:1009E00080BDC04680B588B000AFF860B9607A605D
:1009F0000023FB61A0239B03BB6101237B61164B9A
:100A0000181C012102F006FCBA697B690020111C48
:100A10001A1C04F029F8114B104A926810490A4038
:100A2000802149000A439A600C4B0C4A92680121CC
:100A30000A439A60FB68DAB2BB68101C191C0422D6
:100A4000002303F0F3F97B68181C00F01FF8FB6922
:100A5000181CBD4608B080BD0062040000C00C40F8
:100A6000FFF8FFFF80B582B000AF7860064B181C1E
:100A7000012102F0CFFB7B68181C0B2102F0B2FDB4
:100A8000BD4602B080BDC0460023020080B584B0E0
:100A900000AF78600C23FA18204B111C1A1C03239A
:100AA000081C111C1A1C0AF00DF91D4B181CFFF72D
:100AB000D9FF1C4B181C022102F000FB194B181C1B
:100AC000012102F0A7FB0C23FB1800221A700C2353
:100AD000FB1800225A700C23FB1801229A700C2379
:100AE000FB18181C04F064F80E4B181C02F0ECFB09
:100AF000031C181C796809F0D5FC031C013B1B0280
:100B00001B0A0020191C04F005F804F077F80120F6
:100B100004F024F8BD4604B080BDC04680B5000096
:100B200002001A006006100080B582B000AF021CFF
:100B30003960FB1D1A70FB1D1B78002B0DD0FB1DAF
:100B40001B78012B09D0FB1D1B78022B05D0FB1D48
:100B50001B78032B01D0FB1D1B780949FB1D1A785C
:100B60003B6801209840031C181C131CDB009B18D9
:100B70009B00CB1810335860BD4602B080BDC04604
:100B80000060004080B582B000AF021C3960FB1DE0
:100B90001A70FB1D1B78002B0DD0FB1D1B78012B41
:100BA00009D0FB1D1B78022B05D0FB1D1B78032BE6
:100BB00001D0FB1D1B780949FB1D1A783B680120F9
:100BC0009840031C181C131CDB009B189B00CB18BF
:100BD00010331860BD4602B080BDC04600600040C2
:100BE00080B588B000AF7860344B181C012102F04A
:100BF00011FB7B681B68324A93425BD1314BBB616E
:100C0000BB69181C012102F005FB7B681A797B681F
:100C10005B79101C191C0A22012303F007F97B6879
:100C20009A797B68DB79101C191C0A22012303F0D6
:100C3000FDF80023FB6112E07B681A797B685B7921
:100C4000101C191CFFF79EFF7B681A797B685B7983
:100C5000101C191CFFF768FFFB690133FB61FB697E
:100C6000082BE9DD7B681B687A68127A1202111C76
:100C700003220A439A630823FB1801221A700823EF
:100C8000FB1801225A707B681A690823FB189A60C6
:100C90007B68DA680823FB185A607B681A7D082392
:100CA000FB181A737B681A680823FB18101C191CA0
:100CB00003F024FABD4608B080BDC0464081040060
:100CC00000A0004000B2040090B585B000AF78608D
:100CD0003960144BBB600F23FC187A683B68101C0A
:100CE000191C03F03BFC031C237007E00F23FC18C6
:100CF0007B68181C03F030FA031C23700F23FB18C9
:100D00001B785BB2012B04D1BB685A1EBA60002B62
:100D1000ECD10F23FB181B785BB2181CBD4605B045
:100D200090BDC046E093040080B582B000AF021CC5
:100D3000FB1D1A70064BFA1D1278111C1F220A4067
:100D4000012191400A1C1A60BD4602B080BDC04618
:100D500000E100E080B582B000AF021CFB1D1A70FC
:100D60000649FB1D1B781A1C1F23134001229A40C1
:100D7000C0235B00CA50BD4602B080BD00E100E068
:100D800080B500AF024B5B68181CBD4680BDC046F5
:100D90000000084080B582B000AF7860024B7A68EE
:100DA0009A61BD4602B080BD0000084080B582B0A7
:100DB00000AF7860044B044AD2697968C9430A409D
:100DC000DA61BD4602B080BD0000084080B582B047
:100DD00000AF7860044B044AD1697A680A43DA614B
:100DE000BD4602B080BDC0460000084080B582B05C
:100DF00000AF054BDB697B60034B1B697A681340CE
:100E0000181CBD4602B080BD0000084080B586B009
:100E100000AF786000237B6100233B6102F0EEFDB0
:100E2000031CFB6002E07B6901337B617B69032B60
:100E30000ADC17497A69131C9B009B18DB00CB184E
:100E400018339B79002BEED17B69042B02D1114B17
:100E50003B6114E07B68002B0FD00D497A69131CAD
:100E60009B009B18DB00CB18183301229A717A691A
:100E70007B681A6000233B6101E0074B3B61FB6824
:100E8000181C02F0C9FD3B69181CBD4606B080BDA8
:100E9000300E0020011000F0041000F080B500AF0B
:100EA000204B1B78002B01D0002338E01D4B012282
:100EB0001A701D4B181C012102F0ACF91B4B181CB9
:100EC000022102F08FFB1A4B181C082102F0F6F8E1
:100ED000174B181C012102F09DF9164B181C03F04A
:100EE00067FE0720FFF762FF0720FFF753FF03F0BD
:100EF00085FE0C20FFF72EFF0C20FFF715FF0E4B91
:100F0000181C0021A02209F0E6FE0C4B00221A70EA
:100F10000B4B00221A700B4B00221A600023181C86
:100F2000BD4680BDDA0E00200023020002001A0038
:100F30006006100084B50000300E0020D80E00209E
:100F4000D90E0020D40E0020B0B592B000AFF861E9
:100F50007A613B610B2310229446BC4463440A1C13
:100F60001A700023FB63FB69032B01D9CF4B99E176
:100F700002F044FD031CBB63CD49FA69131C9B00BE
:100F80009B18DB00CB1818339B7901225340DBB24E
:100F9000002B05D0BB6B181C02F03EFDC54B81E158
:100FA0007B69002B0ED13B69002B05D0F969BA6D26
:100FB0003B69081C111C9847BB6B181C02F02CFDE8
:100FC00000236FE1FFF7DCFE031C3B64B849FA69BC
:100FD000131C9B009B18DB00CB1818333A691A606E
:100FE0007B69BB600023FB60B868F968031C5B0C7D
:100FF0000A1CD5031D43031CDC03FA221201002343
:10100000A4185D41231C2C1C181C211CFA2252011F
:10101000002309F0E7FB031C0C1C191C221CA44C28
:10102000F869031C9B001B18DB00E31808331960E8
:101030005A600B2310229446BC4463441B78012B56
:1010400027D17B69FA2292005A43111C9848FA6909
:10105000131C9B009B18DB00C31808335C681B68DB
:101060001A1CF4235343CB1A181C9149FA69131C18
:101070009B009B18DB00CB18103318608C49FA6971
:10108000131C9B009B18DB00CB1810337A225A608C
:1010900018E08749FA69131C9B009B18DB00CB18EA
:1010A00008335C681B6801214942CA17C9186241AC
:1010B0007F4CF869031C9B001B18DB00E318083306
:1010C00019605A607A49FA69131C9B009B18DB006F
:1010D000CB1808335C681B6801210022C9186241E3
:1010E000734CF869031C9B001B18DB00E3181960A4
:1010F0005A606F49FA69131C9B009B18DB00CB18E0
:10110000183301221A716A49FA69131C9B009B1853
:10111000DB00CB1818330B2210218C46BC446244F0
:101120001278DA716249FA69131C9B009B18DB0084
:10113000CB182033BA6D1A605F4B1B78002B05D09B
:10114000BB6B181C02F068FC0023ABE05B4B1B6818
:10115000013304D0594B1B685A1C584B1A60584B2A
:101160001B7801225340DBB2002B35D03B6C1B02B5
:101170001A0A544B1A600220FFF70CFE4C49FA6918
:10118000131C9B009B18DB00CB185C681B683B633F
:101190007C634D4BFB62FB6A3B6000237B603B6BD7
:1011A0007C6B39687A68A24202D803D1994201D98E
:1011B000191C221C0B1CBB623A6CBB6AD3181B02A5
:1011C0001B0A0020191C03F0A5FC0220FFF7FEFDFE
:1011D0003B4B01221A7057E0384B1B68012B53D14F
:1011E0003349FA69131C9B009B18DB00CB1818339A
:1011F00000221A710220FFF7D9FD3B6C1A02314B15
:101200001B681B02D31A1B0A7B647B6C2F4A934218
:1012100001D100237B647B6C181C00F0B9F800F04E
:1012200019FAFB6B002B09D12149FA69131C9B00A9
:101230009B18DB00CB18183301221A71FB6B0133AA
:10124000FB633B6C181C00F037FAFFF799FD031C99
:101250003B643B6C1A021B4B1B681B02D31A1B0A14
:101260007B64002003F03AFC031C1A02154B1B6838
:101270001B02D31A1B0A7B62114B1B78002B03D075
:101280007A6C7B6A9A42B5D80C4B1B68002B04D051
:101290000A4B1B685A1E094B1A60BB6B181C02F0E4
:1012A000BBFB0023181CBD4612B0B0BD021000F0FD
:1012B000300E0020031000F0D80E0020D40E0020C5
:1012C000D90E0020D00E00209BFFFF00FFFFFF0083
:1012D00080B586B000AF02F091FB031C3B61FFF7C5
:1012E00085FD031CFB60FB6803229343181CFFF77A
:1012F00051FDFB68022213403DD0224B01221A709F
:10130000FFF73EFD031C7B610220FFF74FFD7B6969
:101310001A021D4B1B681B02D31A1B0ABB60BB6859
:10132000181C00F035F800F095F97B69181C00F0E6
:10133000C3F9FFF725FD031C7B617B691A02124B81
:101340001B681B02D31A1B0ABB60002003F0C6FBFC
:10135000031C1A020C4B1B681B02D31A1B0A7B606E
:101360000A4B1B78002B03D0BA687B689A42CBD813
:10137000044B00221A703B69181C02F04DFBBD465D
:1013800006B080BDD80E0020D00E0020D90E00205F
:10139000F0B589B000AF78610023FB6150E1AC4C3F
:1013A000F869031C9B001B18DB00E31818330020AE
:1013B0005871A74CF869031C9B001B18DB00E3184D
:1013C00018331B79002B00D137E1A14CF869031CBD
:1013D0009B001B18DB00E3185C681B687869011C24
:1013E0000020021C944202D81ED18B421CD9984C7A
:1013F000F869031C9B001B18DB00E3185C681B6882
:101400007869B8600020F860BD68FE685B1BB44175
:10141000251C1C1C8E4EF869031C9B001B18DB004E
:10142000F3181C605D6008E1894CF869031C9B009F
:101430001B18DB00E3181833DB79002B0AD1844C2E
:10144000F869031C9B001B18DB00E318183300200D
:101450001871DDE07E4CF869031C9B001B18DB0053
:10146000E31808335C681B6878693860002078608E
:101470003D687E685B1BB4411D1C261C744CF869DA
:10148000031C9B001B18DB00E3185C681B68ED184D
:1014900066412C1C351C6E4EF869031C9B001B1802
:1014A000DB00F3181C605D60694CF869031C9B004D
:1014B0001B18DB00E31810331B68002B54DD644C51
:1014C000F869031C9B001B18DB00E31810335C68F1
:1014D0005F4DF869031C9B001B18DB00EB181033F1
:1014E0001B68E4185A4DF869031C9B001B18DB00AD
:1014F000EB1810335C60564CF869031C9B001B18FA
:10150000DB00E31810335B68F32B00D880E0504C0D
:10151000F869031C9B001B18DB00E3185C681B6860
:10152000012500265B197441251C1C1C484EF869D6
:10153000031C9B001B18DB00F3181C605D60444C0F
:10154000F869031C9B001B18DB00E31810335B6871
:10155000F43B1C1C3E4DF869031C9B001B18DB0070
:10156000EB1810335C6053E0394CF869031C9B00A6
:101570001B18DB00E31810335C68354DF869031C59
:101580009B001B18DB00EB1810331B68E41A304D6E
:10159000F869031C9B001B18DB00EB1810335C6020
:1015A0002B4CF869031C9B001B18DB00E31810335D
:1015B0005B68F32B2CD9264CF869031C9B001B1885
:1015C000DB00E3185C681B6801256D42EE175B19B0
:1015D0007441251C1C1C1E4EF869031C9B001B1823
:1015E000DB00F3181C605D60194CF869031C9B005C
:1015F0001B18DB00E31810335B68F43B1C1C144D14
:10160000F869031C9B001B18DB00EB1810335C60AF
:101610000F4CF869031C9B001B18DB00E318183300
:101620001B68002B09D00A4CF869031C9B001B188F
:10163000DB00E318183301205871FB690133FB61AB
:10164000FB69032B00DCAAE6BD4609B0F0BDC0462D
:10165000300E002090B583B000AF00237B6022E005
:1016600014497A68131C9B009B18DB00CB181833B5
:101670005B79002B14D00F497A68131C9B009B18D0
:10168000DB00CB1818331C6878680A497A68131C89
:101690009B009B18DB00CB1820331B68191CA0474C
:1016A0007B6801337B607B68032BD9DDBD4603B0CB
:1016B00090BDC046300E0020F0B58BB000AF786012
:1016C00001235B42DC17BB61FC6100237B622AE0E3
:1016D00039497A6A131C9B009B18DB00CB1818331E
:1016E0001B79002B1CD034497A6A131C9B009B1871
:1016F000DB00CB185C681B68FA69A24205D8FA695E
:10170000A2420DD1BA699A420AD92B497A6A131CAE
:101710009B009B18DB00CB185C681B68BB61FC61FD
:101720007B6A01337B627B6A032BD1DD234B002272
:101730001A70BB69013302D1FB69013338D0BB6930
:10174000FC693B617C611E4BFB60FB681D1C002338
:101750001E1C39697A692B1C341C944202D803D1AF
:101760008B4201D90B1C141CBB61FC61154B1B780F
:1017700001225340DBB2002B05D07B681B021A0A02
:10178000114B1A6002E0104B7A681A600220FFF7D2
:1017900001FBBA697B68D3181B021B0A0020191CC5
:1017A00003F0B8F9054B01221A700220FFF70EFB77
:1017B000BD460BB0F0BDC046300E0020D90E002053
:1017C0009BFFFF00D80E0020D00E002080B582B015
:1017D00000AF021CFB1D1A700649FB1D1B781A1C6A
:1017E0001F23134001229A40C0235B00CA50BD460C
:1017F00002B080BD00E100E080B500AF024B5B6845
:10180000181CBD4680BDC0460000084090B58BB096
:1018100000AF2723FB1800221A702623FB18002292
:101820001A702523FB1800221A702423FB180022AB
:101830001A702323FB1800221A703A1C6C4B111CDF
:101840001A1C0323081C111C1A1C09F03BFA002364
:10185000FB610023BB6100237B6100233B61654B7F
:101860001B6C0422134008D1634B181C012101F0AA
:10187000D1FC2623FB1801221A700F23FC185F4BA2
:10188000181C01F0C1FD031C23700F23FB181B78EB
:10189000032B03D02423FB1801221A70554BDB6A5B
:1018A0004022134003D12323FB1801221A70534B0B
:1018B000181C032101F096FE514B181C01F092FBFD
:1018C000031CBB604E4A80235B00101C191C01F0F6
:1018D000F5FB484B9B6D0122134008D1484B181C67
:1018E000012101F097FC2523FB1801221A7002F058
:1018F00085F8031C7B60434B1B68012213401BD0FF
:10190000404B1B68FB613F4B9B68BB613D4BDB68F9
:101910007B613C4BDB693B613A4B00221A60394BDF
:101920000022DA61374B07229A610C20FFF74EFF45
:101930002723FB1801221A703B1C00229A703B1CC3
:10194000181C03F035F900F079F87B68181C02F0D8
:1019500063F82723FB181B78002B18D0284ABB6894
:10196000101C191C01F0AAFB012003F00BF9254BF8
:10197000BA699A60234B7A69DA60224BFA691A6075
:10198000204B3A69DA61002003F0FCF802E0002005
:1019900003F0E4F82523FB181B78002B04D0184B28
:1019A000181C002101F036FC2423FB181B78002BA7
:1019B00007D0124A0F23FB181B78101C191C01F0CA
:1019C00011FE2323FB181B78002B04D001200021DB
:1019D000002201F089FF2623FB181B78002B04D07E
:1019E000054B181C002101F015FCBD460BB090BD45
:1019F00088B5000000800C400023020002001A009D
:101A0000600610000000084080B582B000AF78602A
:101A10007B680949002B0CD0013B8822120200325E
:101A200053430A68D80AD20A5043800901D00138CA
:101A3000FDD8BD4602B080BD1400002080B584B042
:101A400000AF0823BB60334B802252011A601DE0B7
:101A500000F062F8031C7B60C04600F05DF8021ED7
:101A60007B689A42F9D000F057F8031C7B60294B41
:101A70001B68181C00F058F800F04EF8021C7B6838
:101A8000D31A7B607B68002B00D005E0214B1B68DC
:101A90005B00204A1360DBD11E4B1B685A081D4BAC
:101AA0001A601C4B1B68FB6026E01A4B1A68FB6827
:101AB0001A43184B1A6000F02FF8031C7B60C046D5
:101AC00000F02AF8021E7B689A42F9D000F024F850
:101AD000031C7B600F4B1B68181C00F025F800F0FE
:101AE0001BF8021E7B689A4206D0FB68DA43094B5A
:101AF0001B681A40074B1A60BB685A1EBA60002B5D
:101B000005D0FB685B08FB60FB68002BCDD1BD46B0
:101B100004B080BD1400002080B500AFFFF76CFE5C
:101B2000031C181CBD4680BD80B582B000AF786034
:101B30007B68013BFDD8BD4602B080BD80B586B054
:101B400002AF78602D4B1B78002B01D0002351E0B1
:101B5000FEF7E6FB031CFB60FB68002B01D0FB6873
:101B600048E0274B0020191CFEF704FC031CFB6017
:101B7000FB68002B01D0FB683CE0224B181C00F0F6
:101B80004DFA031CFB60FB68002B01D0FB6831E0C1
:101B90001C4B1B68002B01D10B232BE0184B5B68FF
:101BA0009AB2194B1A80164BDB689AB2164B5A80C0
:101BB000154B00229A80144B0022DA80124B1A88AF
:101BC000114B1A81104B5A880F4B5A810B4B012233
:101BD0001A700D4B1B881A1C0B4B5B8853431A1C45
:101BE000002300930192002000210022002300F036
:101BF0007BF80023181CBD4604B080BDDB0E00201E
:101C0000DC0E0020080F00200C0F002080B582B0F1
:101C100000AF7860084B1B7801225340DBB2002BE9
:101C200001D0012303E07B68044A1A600023181CDA
:101C3000BD4602B080BDC046DB0E00200C0F002068
:101C4000B0B582B000AF051C0C1C101C191CBB1DCC
:101C50002A1C1A803B1D221C1A80BB1C021C1A80E5
:101C60003B1C0A1C1A801E4B1B7801225340DBB21E
:101C7000002B01D001232EE0BB1D1A88BB1C1B8842
:101C8000D318184A1288934208DC3B1D1A883B1C63
:101C90001B88D318134A5288934201DD04231AE0AB
:101CA000BB1C1B88002B03D03B1C1B88002B01D1C5
:101CB000052310E00B4BBA1D12889A80094B3A1D80
:101CC0001288DA80074BBA1C12881A81054B3A1C1D
:101CD00012885A810023181CBD4602B0B0BDC04610
:101CE000DB0E00200C0F0020B0B58CB000AF051C3F
:101CF0000C1C101C191CBB1D2A1C1A803B1D221C0D
:101D00001A80FB1C021C1A70BB1C0A1C1A70BE4BEA
:101D10001B7801225340DBB2002B01D001236EE17E
:101D2000BA4B1B68002B01D1012368E1B84B5B7CE7
:101D3000002B01D00A2362E100237B62B44B9B6835
:101D4000DB083B62B24B1B7C012B02D1BB1C1B7816
:101D500004E0BB1C1B785A425341DBB2FB61FB69B8
:101D6000002B01D0FF2200E000221B23FB181A7079
:101D7000A84BD9883B1D3A1D12888A181A80A34B9C
:101D80001B683A1D1288396A4A439B187B6130E10F
:101D9000A04B1B891A1CBB1D1B88D31A7A6C93425B
:101DA00000D9131CFB627A6CFB6AD31A7B64994BD3
:101DB0009988BB1DBA1D12888A181A807B6A3A6AF4
:101DC00053431A1C7B699B18BB62FB6A072B5BD8C9
:101DD000BB1D1B88FA6AD318FB62FB69002B28D055
:101DE00021E0BB1D1B88DB089BB21A1CBB6A9B1839
:101DF000BA1D1288D20892B2111CBA6A521812780F
:101E0000D0B2BA1D128807210A40012191400A1C54
:101E1000D2B2011C0A43D2B2D2B21A70BB1D1A88C8
:101E2000BB1D01321A80BB1D1A88FB6A9A42D8D3A7
:101E3000BFE023E0BB1D1B88DB089BB21A1CBB6AFA
:101E40009B18BA1D1288D20892B2111CBA6A521895
:101E50001278D0B2BA1D128807210A4001219140A0
:101E60000A1CD2B2D243D1B2021C0A40D2B2D2B2C0
:101E70001A70BB1D1A88BB1D01321A80BB1D1A883F
:101E8000FB6A9A42D6D394E0BB1D1B8807221340FD
:101E90003B61BB1D1B88DB089BB21A1CBB6A9B18ED
:101EA000BB623B69002B37D00F23FB18BA6A12784C
:101EB0001A7001223B699A40131CDAB20E23FB18F8
:101EC000013A1A700F23FB180F22BA180E21791845
:101ED000127809780A401A700E23FB181B78DB432E
:101EE000D9B21B23FB181A780B1C1340DAB20F234C
:101EF000FB181B781343DAB20F23FB181A70BB6A66
:101F00000F22BA1812781A70BB6A0133BB623A69A1
:101F1000FB6AD318083BFB62FB6ADB08BB60BB684B
:101F2000002B13D01B23FB181A78BB68B96A081C56
:101F3000111C1A1C08F0CFFEBB68DB001A1CFB6AE0
:101F40009B1AFB62BB68BA6AD318BB62FB6A002BA0
:101F50002FD00F23FB18BA6A12781A70FB6A01227D
:101F60009A40131CDAB20E23FB18013A1A700E23A2
:101F7000FB181B78DB43D9B20F23FB181A780B1C14
:101F80001340DAB20F23FB181A701B23FB180E2222
:101F9000BA181B7812781340D9B20F23FB180F22FE
:101FA000BA1812780A431A70BB6A0F22BA1812784C
:101FB0001A703B1D1A887B6AD3185A113B1D198869
:101FC0007B6ACB185911144B8900CB58391D0888EE
:101FD000796A41181F20014001208840011C1943E3
:101FE0000D4B9200D150BB1D00221A807B6A013339
:101FF0007B627B6C002B00D0CAE6C0460023181C15
:10200000BD460CB0B0BDC046DB0E0020080F00205E
:10201000DC0E00200C0F0020880F002090B583B04C
:1020200000AF78600E4B9C690D4B59680C4BDA6819
:102030000B480C4BA0470B4B1B68002B01D10B230B
:102040000AE0084B1A687B681A60074B181CFF21CE
:10205000102208F040FE0023181CBD4603B090BDBE
:10206000DC0E0020080F0020880F0020B0B58AB0D9
:1020700002AF424B9B68DB08FB60414B1B687B61F6
:1020800001233B610023FB610023BB6143E07B69CB
:102090000122134003D0BB690133BB612AE0BB6955
:1020A000002B24D0374B1A68FB68F9694B43D318CF
:1020B000BB60324B1C6A314B5D683049BA68FB69C2
:1020C0000093BB690193081C111C00222B1CA04724
:1020D000031C7B607B68002B01D07B6849E0BA69F8
:1020E000FB69D3180133FB610023BB6102E0FB698C
:1020F0000133FB61FA69BB69D3181F22134003D077
:102100007B695B087B6106E03B695A1C3A611C4AAB
:102110009B009B587B61FA69BB69D218174BDB683F
:102120009A42B4D3BB69002B1CD0164B1A68FB68CB
:10213000F9694B43D318BB60104B1C6A0F4B5D68A9
:102140000E49BA68FB690093BB690193081C111C16
:1021500000222B1CA047031C7B607B68002B01D056
:102160007B6806E0064B181C0021102208F0B3FD26
:102170000023181CBD4608B0B0BDC046DC0E0020D0
:10218000880F0020080F002080B584B000AFF860F1
:10219000B9607A603B60FB681B0CDAB2BB681A70EE
:1021A000FB681B0ADAB27B681A70FB68DAB23B681C
:1021B0001A70BD4604B080BD80B588B000AF7860AD
:1021C0007B68002B01D105233DE07B6800225A602B
:1021D0007B681F4A9A601823FB18181CFFF716FD2E
:1021E000031CFB61FB69002B01D0FB692BE0BA6982
:1021F0007B681A600823FB1800221A600823FB186A
:1022000000225A60BB691B885A1E0823FB189A607B
:10221000BB695B885A1E0823FB18DA607A680823BA
:10222000FB18101C191C00F017F8031CFB61FB695C
:10223000002B01D0FB6906E07A68064B101C191CC4
:1022400000F038FBFB69181CBD4608B080BDC046D5
:10225000FFFFFF00ACB8000090B589B000AF786018
:1022600039607B68002B02D03B68002B01D105232D
:1022700069E03B681A683B689B689A4205DA3B68EC
:102280005A683B68DB689A4201DB04235BE03B68E9
:102290001A687B681B689B889A4216DB3B685A6801
:1022A0007B681B68DB889A420FDB3B689A687B6817
:1022B0001B681B89013B9A4207DC3B68DA687B6834
:1022C0001B685B89013B9A4201DD03233BE03B68CD
:1022D0001B6898B23B685B6899B23B681B689AB20E
:1022E0003B689B689BB2D3189BB201339CB23B689E
:1022F0005B689AB23B68DB689BB2D3189BB2013330
:102300009BB2221CFFF79CFC031CFB613B681A6814
:102310000C23FB181A603B685A680C23FB185A60A0
:102320003B689A680C23FB189A603B68DA680C23B8
:10233000FB18DA607B680C22BA180C3313CA13C37B
:1023400012681A60FB69181CBD4609B090BDC046F2
:10235000B0B588B002AF78607B68002B01D105234F
:1023600031E07B6858680B23F9180A23FA1809230F
:10237000FB1800F045F87B68181C00F029F8031CD6
:102380007B617B69002B01D07B691CE07B681B684B
:102390001B893B617B681B685B89FB600B23FB1817
:1023A0001D780A23FB181C780923FB181A783B694F
:1023B000F9684B4300920193002000212A1C231C42
:1023C000FFF792FC031C181CBD4606B0B0BDC0460A
:1023D00080B582B000AF78607B68002B01D1052307
:1023E0000AE07B681B681A887B681B685B88002092
:1023F0000021FFF725FC031C181CBD4602B080BD60
:1024000080B584B000AFF860B9607A603B60F8686E
:10241000B9687A683B68FFF7B7FEBD4604B080BD77
:1024200090B589B002AFF860B9607A60FB68002BA4
:1024300001D1052330E0FB680C33191CBA687B68B6
:10244000081C111C1A1C00F06BF8031C1A1C012339
:102450005340DBB2002B01D001231DE0FB689868DC
:102460001723F9181623FA181523FB18FFF78CFE0B
:10247000BB6898B27B6899B21723FB181A781623A9
:10248000FB181C781523FB181B780093012301937C
:10249000231CFFF729FC031C181CBD4607B090BD88
:1024A00090B589B002AFF860B9607A603B60FB68B4
:1024B000002B01D105232FE0FB680C33191CBA68EF
:1024C0007B68081C111C1A1C00F02AF8031C1A1C3B
:1024D00001235340DBB2002B01D001231CE03868FC
:1024E0001723F9181623FA181523FB18FFF74CFECB
:1024F000BB6898B27B6899B21723FB181A78162329
:10250000FB181C781523FB181B78009301230193FB
:10251000231CFFF7E9FB031C181CBD4607B090BD48
:1025200080B584B000AFF860B9607A60FB68002BBA
:1025300013D0FB681A68BB689A420EDCFB689A6885
:10254000BB689A4209DBFB685A687B689A4204DCE4
:10255000FB68DA687B689A4201DA002300E0012315
:10256000181CBD4604B080BD80B58CB000AFF860CB
:102570007A603B600B23FB180A1C1A7000237B62F5
:10258000FB68002B01D1052328E10B23FB181B78E6
:102590001F2B04D90B23FB181B787E2B01D9022398
:1025A0001CE1FB6828229B5C022B1AD10B23FB1831
:1025B0001B789AB22E23FB18303A1A800B23FB1893
:1025C0001B783A2B03D12E23FB180A221A800B23E7
:1025D000FB181B78202B0CD12E23FB180B221A8002
:1025E00007E00B23FB181B789AB22E23FB18203A26
:1025F0001A802E23FB181A88FB681B8C013B9A4219
:1026000001DD0223EAE0FB68DB693B62FB68DB6912
:10261000FB61FB68DB69BB612C23FB1800221A807D
:10262000CEE0FB6822229B5C012B02D0022B0AD059
:1026300014E02E23FB181B883A6AD3181A782A2331
:10264000FB181A8014E02E23FB181B885B00FA6924
:10265000D2182A23FB1812881A8009E02E23FB18AF
:102660001B889B00BA69D3181A682A23FB181A80A2
:102670002823FB1800221A8051E02A23FB181B880C
:10268000012213401CD02823FB181A887B68D1181C
:102690002C23FB181A883B68D318FA68101C1A1CE4
:1026A000FFF7BEFE031C7B617B69012B01D97B69AF
:1026B00094E07B69002B24D17B6A01337B6220E0AC
:1026C0003823FB181B78002B1BD02823FB181A88F3
:1026D0007B68D1182C23FB181A883B68D218FB683A
:1026E0005B68F868FFF7DCFE031C7B617B69012BEC
:1026F00001D97B6972E07B69002B02D17B6A0133CF
:102700007B622A23FB182A22BA18128852081A80E0
:102710002823FB182822BA18128801321A80FB6875
:1027200024229B5C9BB22822BA1812889A42A4D316
:1027300027E03823FB181B78002B1BD02823FB181D
:102740001A887B68D1182C23FB181A883B68D2188A
:10275000FB685B68F868FFF7A3FE031C7B617B697D
:10276000012B01D97B6939E07B69002B02D17B6A9F
:1027700001337B622823FB182822BA181288013201
:102780001A802823FB181A88FB6824215B5C181C1C
:10279000FB6827215B5CC3189A42CADBFB682322D3
:1027A0009B5C99B22E23FB182E22BA1812888A1825
:1027B0001A802C23FB181A882C23FB1801321A804C
:1027C000FB6825229B5C9BB22C22BA1812889A4285
:1027D00000D226E77B6A5A425341DBB2181CBD4641
:1027E0000CB080BD90B58DB002AFF860B9607A6072
:1027F0003B6000237B62FB68002B02D0BB68002B90
:1028000001D1052352E0FB6828229B5C002B01D1FB
:1028100002234BE03B68FB61BB6BBB6100233B6267
:102820003CE0BA683B6AD3181B780A2B0DD13B6891
:10283000FB61FB6825229B5C1A1CBB69D318FA68F4
:102840002621525C9B18BB6125E0BA683B6AD3180D
:102850001978F868FA69BC693C23FB181B78009367
:10286000231CFFF781FE031C7B617B69012B01D9CF
:102870007B691BE07B69002B02D17B6A01337B62A1
:10288000FB6824229B5C191CFB6827229B5CCB18ED
:10289000FA69D318FB613B6A01333B623A6A7B6891
:1028A0009A42BED37B6A5A425341DBB2181CBD46E2
:1028B0000BB090BD80B582B000AF786039607B68A6
:1028C000002B01D1052315E03B68002B08D17B6864
:1028D0001C33181C0021102208F0FDF9052309E023
:1028E0007B681C331A1C3B68101C191C102208F052
:1028F000E9F90023181CBD4602B080BD80B586B042
:1029000000AF7860081C111CFB1C021C1A70BB1C59
:102910000A1C1A70BB1C1B78002B04D01023FB6010
:10292000394B3B6103E00023FB60384B3B617B6824
:102930005B6B3A691340BB6000237B61FB1C1B7817
:10294000062B54D89A00324BD3181B689F46314B44
:102950005A68FE23DB0113407A6913437B612D4BD8
:102960005B687F2213407A6913437B6142E0294B05
:102970005A68FE23DB0513401B0E1B027A691343C2
:102980007B61244B5A68FE23DB0313401B0C7A69DE
:1029900013437B612EE01F4B9A68FE23DB0113403B
:1029A0007A6913437B611B4B9B687F2213407A69D2
:1029B00013437B611EE0174B9A68FE23DB0513402F
:1029C0001B0E1B027A6913437B61124B9A68FE232C
:1029D000DB0313401B0C7A6913437B610AE00D4B48
:1029E000DB687F2213407A6913437B6102E0002396
:1029F0007B61C046FB687A699A40BB681A437B6872
:102A00005A63BD4606B080BDFFFF80808080FFFF17
:102A1000BCB80000B081E00F90B585B000AF786021
:102A200039600B23FB183A6812791A700B23FB18D4
:102A30001B78002B09D10B23FC181F4B181C0021FD
:102A400000F08CF8031C23700AE01B4B181C0021BB
:102A500000F084F8FA23DB01181C002100F07EF856
:102A60007B680A225A603B681B781A063B68DB7851
:102A70001904FE23DB030B401A430B23FB181B78BE
:102A80001902FE23DB010B401A433B685B781B01F4
:102A900013433A6892781343FB603B685B79002BE1
:102AA00003D0FB6808221343FB607B68FA681A6056
:102AB000BD4605B090BDC046405DC60080B584B03F
:102AC00000AF786039607B6802225A603B689B786F
:102AD0007A68101C191C0022FFF710FF3B681B7856
:102AE0001A073B685B781B051A433B681B791B027E
:102AF00013431A1C3B68DB781B011343FB603B68E4
:102B00009B79002B04D0FB68802252041343FB60A6
:102B10003B68DB79002B03D0FB6804221343FB6086
:102B20003B685B79002B03D0FB6802221343FB60F8
:102B30003B681B7A002B03D0FB6801221343FB6028
:102B40003B689B781B041A1CFB681343FB607B6883
:102B5000FA68DA60BD4604B080BDC04680B584B076
:102B600000AF786039607B68154A934202D9144BF4
:102B70007B6006E07B68134A934202D8FA23DB01AC
:102B80007B603B68002B05D10F4B181C00F09CFBB1
:102B9000031C3B603A687B68D318013B181C7968BA
:102BA00007F080FC031CFB60FB68002B02D0FB6875
:102BB000013BFB60FB68DBB2181CBD4604B080BD66
:102BC000405DC600FF7C00004081040080B582B0FB
:102BD00000AF78607B68002B0AD10F4B181C00F007
:102BE00073FB031C7B607B68002B01D101237B609E
:102BF0007B680A4A944663447B607B68181C0849DA
:102C000007F050FC031C7B607B68DBB2013BDBB24E
:102C1000181CBD4602B080BD408104003F420F0039
:102C200040420F0080B586B000AFF860B9607A60AE
:102C3000FB681B687B61BB6801229A40131CDB4365
:102C40001A1C7B691A407B6801211940BB689940B6
:102C50000B1C1A43FB681A60BD4606B080BDC04617
:102C600080B582B000AF786039607B681A683B68D5
:102C7000DA40131C01221340181CBD4602B080BD6F
:102C800080B584B000AF78607B68002B05D07A688F
:102C900080231B029A4200D8C046786807F084FD62
:102CA000031C1A1C1F239B1AFB60FB68181CBD46E3
:102CB00004B080BD80B582B000AF78607B6801222F
:102CC0009A40131C181CBD4602B080BD80B500AFF1
:102CD000034BDB6C1B0EDBB2181CBD4680BDC0462F
:102CE000B081E00F80B582B000AF224B5A69E0237B
:102CF000DB0013408022920093421ED0802292007B
:102D0000934206D8002B26D08022520093421FD037
:102D100027E0C0229200934204D0E022D2009342E6
:102D20001CD01EE0FFF7D2FF031E122B02D9124B5C
:102D30007B6019E0114B7B6016E0FFF7C7FF031EB5
:102D4000122B02D90E4B7B600EE00E4B7B600BE02A
:102D50000D4B7B6008E00D4B7B6005E00C4B7B600E
:102D600002E000237B60C0467B68181CBD4602B0B1
:102D700080BDC04600800C40804F120040420F00D2
:102D800040B56400C0CF6A00C0D8A700809FD500BE
:102D9000406F400190B583B000AFFC1C0E4B181C77
:102DA00000F032FB031C2370FB1C1B78072B06D0A2
:102DB000082B09D1FDF716FA031C7B6007E0FFF72B
:102DC00091FF031C7B6002E000237B60C0467B68B0
:102DD000181CBD4603B090BD06000C0080B584B041
:102DE00000AF7860174BDA6B0B23FB18511E8A413A
:102DF0001A70144B144ADA63124B5B6807221340B3
:102E0000FB607B68114A934206D87B68104A934264
:102E100002D90123FB6001E00023FB60094B094A52
:102E2000526807218A43111CFA680A435A600B232F
:102E3000FB181B78002B02D0024B0022DA63BD4640
:102E400004B080BD00000C40711B00000048E80188
:102E50000024F40080B500AFFDF7BCF9031C181C7A
:102E6000FFF7BCFFBD4680BD80B584B000AF786081
:102E70000023BB607B68364A934206D0354A9342B2
:102E800003D0354A934200D000E0C0467B68181C4E
:102E900000F0BAFA031CFB607B682D4A93420CD009
:102EA0002C4A934210D02C4A934200D013E02B4B73
:102EB0009B6A03221340FB600DE0284B9B6A0C22A7
:102EC00013409B08FB6006E0244B9B6A30221340B2
:102ED0001B09FB60C046FB68012B05D014D3022BF5
:102EE00007D0032B0AD02BE0FDF700FA031CBB60D0
:102EF00029E0FDF70BFA031CBB6024E0FDF74EF957
:102F0000031C5B08BB601EE00023BB607B68124AA9
:102F1000934203D07B680E4A934210D10F4B9A6ABA
:102F20007B680D498B4201D1102300E01423DA4065
:102F3000131E04D0FDF7E2F9031CBB6003E002E0BE
:102F40000023BB60C046BB68181CBD4604B080BDF2
:102F500003001C0004001E0002001A0000800C4048
:102F600080B582B000AF7860074B5B6D01221340E3
:102F700000D005E0C046044B1B6D7A681340FAD1BF
:102F8000BD4602B080BDC04600800C4090B583B005
:102F900000AFFC1C124B181C00F036FA031C237007
:102FA000FB1C1B78032B08D0082B0BD0022B0ED157
:102FB000FDF7ACF9031C7B600CE0FDF797F9031CEF
:102FC0007B6007E0FDF70EF9031C7B6002E0002345
:102FD0007B60C0467B68181CBD4603B090BDC046F0
:102FE0000733220080B584B000AF78607B681B098E
:102FF0000F221340BB60BB68072B4ED8BB689A00FA
:103000002A4BD3181B689F46294B1A68E0235B02A2
:1030100013409B0B0133FB6042E0254B9B680F2262
:103020001340FB60FB68181CFFF744FE031CFB60A9
:1030300036E01F4B5B680F221340FB60FB68181CD7
:10304000FFF738FE031CFB602AE07B68194A9342B5
:103050000BD1174B9B6E0F221340FB60FB68181CB3
:10306000FFF728FE031CFB6002E00123FB60C04663
:1030700016E07B68104A93420BD10D4B1B6F032265
:103080001340FB60FB68181CFFF714FE031CFB6079
:1030900002E00123FB60C04602E00123FB60C04662
:1030A000FB68181CBD4604B080BDC046D8B80000FF
:1030B00000800C40600610007007160080B584B0D8
:1030C00000AF786039607B681B090F221340FB60FA
:1030D000FB68072B00D98FE0FB689A00484BD31898
:1030E0001B689F463B68002B03D03B68082B00D829
:1030F000C046FFF7AFFE434B424A126842491140B7
:103100003A68013A92030A431A60FDF747F8031C34
:10311000BB60BB68181CFFF761FE6EE03B68002BCC
:1031200005D03A6880239B009A4200D8C0463B688D
:10313000181CFFF7A5FD031C3B60324B314A926817
:103140000F218A43111C3A680A439A6055E03B6894
:10315000002B05D03A6880239B009A4200D8C046D5
:10316000FFF778FE3B68181CFFF78AFD031C3B60E5
:10317000244B244A52680F218A43111C3A680A439F
:103180005A60FDF70BF8031CBB60BB68181CFFF707
:1031900025FE32E07B681D4A934200D012E00420F5
:1031A000FFF7DEFE3B68181CFFF76AFD031C3B605F
:1031B000144B144A926E0F218A43111C3A680A4339
:1031C0009A66C04619E07B68114A934200D012E02B
:1031D0004020FFF7C5FE3B68181CFFF751FD031C9C
:1031E0003B60084B074A126F03218A43111C3A685F
:1031F0000A431A67C04600E0C046BD4604B080BD21
:10320000F8B8000000800C40FF3FFEFF6006100091
:103210007007160080B586B000AF78600A1CFB1CF2
:103220001A7000233B617B681B0A0F2213400A2B94
:1032300036D89A001C4BD3181B689F461B4B7B61EA
:1032400018E01B4B7B6115E01A4B7B6112E01A4BB7
:103250007B6101233B610DE0184B7B6110233B61D7
:1032600008E0174B7B6180235B003B6102E0154B5C
:103270007B61C0467B681B0B1F221340FB603B69D0
:10328000002B03D03B69181CFFF76AFEFB1C1B7860
:103290007969FA68081C111C1A1CFFF7C3FC00E0CE
:1032A000C046BD4606B080BD18B9000040800C4045
:1032B00008800C4044800C4058800C4060800C40DA
:1032C00064800C4078800C4080B584B000AF78609A
:1032D0007A68F8239B031340E0221203934200D143
:1032E00079E0E0221203934213D8802292029342A3
:1032F0003BD080229202934202D8002B23D074E06C
:103300008022D202934223D0C022120393425DD086
:103310006BE0D022520393422CD0D022520393422E
:1033200008D88022520393422BD0B02252039342FA
:103330003DD05AE0E0225203934231D088229203DA
:1033400093424DD051E0FCF74DFF031CFB604FE072
:10335000FCF748FF031CFB60284B9B680F221340BF
:103360001A1CFB68D340FB6042E0FCF717FF031C0C
:10337000FB603DE0224B181CFFF776FD031CFB6051
:1033800036E01F4B181CFFF76FFD031CFB601B4B47
:103390009B6E0F2213401A1CFB68D340FB6027E092
:1033A000184B181CFFF760FD031CFB6020E0154B59
:1033B000181CFFF759FD031CFB60104B1B6F032209
:1033C00013401A1CFB68D340FB6011E0FFF7E2FCDE
:1033D000031CFB600CE0FFF785FC031CFB6007E0AF
:1033E000FFF7D4FD031CFB6002E00023FB60C04636
:1033F000FB68181CBD4604B080BDC04600800C4070
:1034000002001A0003001C0080B584B000AF786091
:103410000F23FB1801221A707B680F221340BB6038
:10342000BB68072B00D9CAE0BB689A006A4BD31867
:103430001B689F46694BDB6A694A13408022520130
:10344000934216D080225201934204D88022120166
:10345000934213D01CE080229201934204D0802238
:10346000D20493420FD013E00F23FB1802221A70EC
:1034700013E00F23FB1803221A700EE00F23FB1832
:1034800004221A7009E00F23FB180A221A7004E0C4
:103490000F23FB1805221A70C04695E04F4B9B6A1C
:1034A00003221340022B08D0032B0BD0012B0ED18B
:1034B0000F23FB1803221A7015E00F23FB180222BA
:1034C0001A7010E00F23FB1806221A700BE0434B12
:1034D0009A6A80235B02134004D00F23FB180B224F
:1034E0001A7000E0C0466FE03C4B9B6A0C22134010
:1034F000082B08D00C2B0BD0042B0ED10F23FB185C
:1035000003221A7015E00F23FB1802221A7010E034
:103510000F23FB1806221A700BE0304B9A6A8023A7
:103520005B03134004D00F23FB180B221A7000E03A
:10353000C04649E0294B9B6A30221340102B02D031
:10354000202B05D009E00F23FB1803221A7009E095
:103550000F23FB1802221A7004E00F23FB1801222C
:103560001A70C04630E00F23FB1807221A702BE0B8
:103570001A4BDA6AE023DB02134080229202934264
:1035800012D08022D202934204D08022520293426F
:1035900005D00EE00F23FB1809221A700EE00F234E
:1035A000FB1802221A7009E00F23FB1803221A707D
:1035B00004E00F23FB1801221A70C04604E00F2319
:1035C000FB1800221A70C0460F23FB181B78181C2A
:1035D000BD4604B080BDC04644B9000000800C4028
:1035E000003C000480B588B000AF78600A1CFB1C6A
:1035F0001A700323FB611B23FB1803221A7000239C
:103600003B617B680F221340FB60FB68072B00D9EE
:10361000F2E0FB689A007C4BD3181B689F46FB1CAA
:103620001B780B2B00D9E9E09A00784BD3181B6864
:103630009F460423FB611B23FB1800221A701BE02A
:103640000323FB611B23FB1801221A7014E00223E1
:10365000FB611B23FB1802221A700DE00123FB61A2
:103660001B23FB1803221A7006E00523FB611B23B2
:10367000FB1805221A70C0461B23FB181B78181C68
:103680000121012200F030F9FFF7E4FB604BFA69F9
:103690005A6200F0AFFAFCF781FD031CBB60BB6807
:1036A000181CFFF79BFBACE0FB1C1B780B2B00D915
:1036B000A6E09A00574BD3181B689F4600237B61F6
:1036C0001DE000200121012200F00EF902237B61A0
:1036D00015E001200121012200F006F901237B61A0
:1036E0000DE04D4B181C02210122FFF79BFA03232A
:1036F0007B6104E000237B6101233B61C046FB68E2
:10370000022B0BD1424B424A926A444911407A69DA
:1037100011433A6912040A439A6272E03C4B3C4AF4
:10372000926A3F4911407A69920011433A69120541
:103730000A439A6265E0FB1C1B78022B07D0032B1F
:103740000DD0012B00D05CE000237B610FE0002056
:103750000121012200F0C8F802237B6107E001206B
:103760000121012200F0C0F801237B61C046284BF3
:10377000274A926A30218A43111C7A6912010A434E
:103780009A623EE0FB1C1B78032B14D0092B22D03D
:10379000022B00D035E000200121012200F0A4F826
:1037A0001B4B40225A62C046194BDA6A80235B02E7
:1037B0001340F9D01FE001200121012200F094F80C
:1037C000134B60225A62C046114BDA6A80239B0277
:1037D0001340F9D00FE005200121012200F084F808
:1037E0000B4B80225A62C046094BDA6A8023DB0207
:1037F0001340F9D0C04604E0C04602E0C04600E0F5
:10380000C046BD4608B080BD64B9000084B9000060
:1038100000800C40B4B9000040800C40FCFFFEFF6B
:10382000F3FFEFFF90B587B000AF021CFB1D1A70CD
:10383000FB1D1B78042B4DD89A00284BD3181B680E
:103840009F46274BDB6AFF2213407B611AE0244B23
:10385000DA6AFF231B0213401B0A7B6112E0204B34
:10386000DA6AFF231B0413401B0C7B610AE01C4B2C
:10387000DB6A1B0E7B6105E0194B1B6BFF221340BB
:103880007B61C0461323FC181120FFF7BDFD031C0C
:1038900023701323FB181B78052B01D1FFF7DAFAED
:1038A000104B104AD268D20AD202F91D09780902D7
:1038B00011437A690A43DA601323FB181B78052B3E
:1038C00009D1FCF76BFC031CFB60FB68181CFFF7BD
:1038D00085FA00E0C046BD4607B090BDE4B90000DF
:1038E000B081E00F00800C4090B587B000AF041CA1
:1038F000081C111CFB1D221C1A70BB1D021C1A7017
:103900007B1D0A1C1A70FB1D1B78052B4DD89A00D5
:10391000284BD3181B689F4601233B610223FB60A1
:1039200001237B6126E004233B610823FB60032322
:103930007B611FE010233B612023FB6005237B613B
:1039400018E040233B618023FB6007237B6111E08B
:1039500080235B003B6180239B00FB6009237B612C
:1039600008E08023DB003B6180231B01FB60162302
:103970007B61C046BB1D1B78002B10D00E4B3A69F3
:103980001A627B1D1B78002B0CD0C0460B4A7B694A
:10399000101C191CFFF764F9031EF7D002E0064B58
:1039A000FA681A6200F026F900E0C046BD4607B08A
:1039B00090BDC046F8B9000000800C402C800C403F
:1039C00080B584B000AF78600A1CFB1C1A7000231D
:1039D000FB60FB1C1B78002B01D00123FB607B6884
:1039E0005B005A1C0449FB68081C111C1A1CFFF7D9
:1039F00019F9BD4604B080BD78800C4080B582B016
:103A000000AFEFF310833B603B687B6072B67B686E
:103A1000181CBD4602B080BD80B582B000AF786092
:103A20007B68002B00D162B6BD4602B080BDC046A7
:103A300080B500AFFCF7B2FBBD4680BD80B500AFDE
:103A4000024A84230021D150BD4680BD00800C4035
:103A500080B500AF024A84230249D150BD4680BDE3
:103A600000800C400E58000080B582B000AF494A7B
:103A70008423D358012213407B60FFF7E9FF002322
:103A80003B60454B1B68012213403A6813433B607F
:103A9000414B1B68102213403A6813433B603E4B76
:103AA0001B68402213403A6813433B603A4B1B6843
:103AB000042213403A6813433B60374B1A68802353
:103AC0005B0013403A6813433B60334B1A68802312
:103AD0009B03134002D08023DB0000E000233A6800
:103AE00013433B602B4B3A681A622B4B1B682B4AE3
:103AF000134080225201934211D0802252019342FE
:103B000004D88022120193421ED032E0802292011A
:103B100093420ED08022D20493421FD029E0C046A7
:103B20001C4BDB6A80221340FAD01A4B03225A62E4
:103B30001FE0C046174BDA6A80239B001340F9D080
:103B4000144B04225A6214E0C046124BDB6A08226E
:103B50001340FAD00F4B02225A620AE0C0460D4BC6
:103B6000DA6A8023DB031340F9D00A4B05225A623C
:103B7000C046094B1B680122134002D1054B0222AB
:103B80001A627B68002B01D0FFF758FFBD4602B0D8
:103B900080BDC04600800C40180F0020003C00048F
:103BA00080B582B000AF021CFB1D1A700E4BDA6AA2
:103BB0000E4B1A600E4B0E4A126904210A431A6119
:103BC00030BFFB1D1B78002B02D0FFF74DFF07E035
:103BD000064B1A688023DB00134001D1FFF728FF52
:103BE000BD4602B080BDC04600800C40180F0020CA
:103BF00000ED00E080B500AF024BDA6A024B1A60BC
:103C0000BD4680BD00800C40180F002080B586B0F6
:103C100000AFF860B9607A60FB681B687B61BB68C5
:103C200001229A40131CDB431A1C7B691A407B68F3
:103C300001211940BB6899400B1C1A43FB681A60AC
:103C4000BD4606B080BDC04680B584B000AFF86008
:103C5000B9607A60FB681B68BA68D2431A407B6817
:103C60001A43FB681A60BD4604B080BD80B582B0BF
:103C700000AF021C3960FB1D1A70FB1D1B78002B66
:103C80000DD0FB1D1B78012B09D0FB1D1B78022BCF
:103C900005D0FB1D1B78032B01D0FB1D1B780949A8
:103CA000FB1D1A783B6801209840031C181C131C4C
:103CB000DB009B189B00CB1810335860BD4602B048
:103CC00080BDC0460060004080B582B000AF021CDD
:103CD0003960FB1D1A70FB1D1B78002B0DD0FB1DDE
:103CE0001B78012B09D0FB1D1B78022B05D0FB1D77
:103CF0001B78032B01D0FB1D1B780949FB1D1A788B
:103D00003B6801209840031C181C131CDB009B1807
:103D10009B00CB1810331860BD4602B080BDC04672
:103D20000060004080B586B000AFB9607A60191CB1
:103D30000F23FB18021C1A700E23FB180A1C1A70A2
:103D40000F23FB181B78002B11D00F23FB181B78B7
:103D5000012B0CD00F23FB181B78022B07D00F234D
:103D6000FB181B78032B02D00F23FB181B787B68F2
:103D7000072B11D87B689B001A1C07239340191C42
:103D80000F23FB181B787A68920093401A1C214B72
:103D9000181CFFF759FF13E07B68083B7B617B69C8
:103DA0009B001A1C07239340191C0F23FB181B7838
:103DB0007A69920093401A1C174B181CFFF744FFB6
:103DC0000E23FB181B7815497A68081C111C1A1C55
:103DD000FFF71CFF2023FB181B7811497A68081C89
:103DE000111C1A1CFFF712FF0E4A7B680121994033
:103DF0000B1C191C8E235B00D1502423FB181B784D
:103E000009497A68081C111C1A1CFFF7FFFEBD4601
:103E100006B080BD006100400461004008610040C0
:103E20000C6100400060004010610040B0B584B0FB
:103E300000AFB960111C7B600F23FB18021C1A70C5
:103E40000E23FB180A1C1A700F23FB181B78002B7B
:103E500011D00F23FB181B78012B0CD00F23FB185C
:103E60001B78022B07D00F23FB181B78032B02D0E3
:103E70000F23FB181B780E23FB181B78002B13D085
:103E80007B68002B08D00F23FB181A78BB68101C26
:103E9000191CFFF719FF07E00F23FB181A78BB68FE
:103EA000101C191CFFF7E2FEBB68072B22D8344C0C
:103EB0000F23FB181A7832480F23FB1819780B1CB4
:103EC000DB005B189B00C3185B68B9688900081C9D
:103ED0000F218140C9430B400E2179180978B86839
:103EE000800081401943131CDB009B189B00E318E2
:103EF000596029E0224C0F23FB181A7820480F2321
:103F0000FB1819780B1CDB005B189B00C3180833E7
:103F10001B68B9681B48844661448900081C0F214E
:103F20008140C9430B400E2179180978B868154DB6
:103F3000AC466044800081401943131CDB009B1891
:103F40009B00E318083319600E23FB181B78002B25
:103F500013D17B68002B08D00F23FB181A78BB689D
:103F6000101C191CFFF7B0FE07E00F23FB181A788E
:103F7000BB68101C191CFFF779FEBD4604B0B0BD2C
:103F800000600040F8FFFF3F80B586B000AFF860EA
:103F9000B9607A60FB681B687B61BB6801229A404C
:103FA000131CDB431A1C7B691A407B6801211940F2
:103FB000BB6899400B1C1A43FB681A60BD4606B0EB
:103FC00080BDC04680B584B000AFF860B9607A604B
:103FD000FB681B68BA68D2431A407B681A43FB68C7
:103FE0001A60BD4604B080BD90B589B000AFF860DE
:103FF000B9607A601A1CFB1C1A707B68002B00D118
:1040000066E0FB681B68344A1A40FB681A60FA686D
:10401000FB1C1B781B021C1CC0239B00101C191CC2
:10402000221CFFF7CFFFBB68002B05D12B4B181CC0
:10403000FFF74AF9031CBB6001235B42BB61FB68CD
:104040001B680222134012D0FB1C1B78012B07D0E7
:10405000022B08D0002B00D01AE0214BBB6105E0F9
:10406000204BBB6102E0204BBB61C04610E0FB1C53
:104070001B78012B06D0022B07D0002B08D11B4B3D
:10408000BB6105E01A4BBB6102E01A4BBB61C04645
:10409000FB1C1B78184AD35C7B617B689B00BA6869
:1040A000D11A7B697A685343081C191C06F0FAF987
:1040B000031C013BFB61FB681B680222134004D018
:1040C000FB69002B01D10123FB61FA69FB681A61CE
:1040D000BD4609B090BDC046FFFCFFFF4081040013
:1040E00040164000C0D8A7008050740180841E0094
:1040F00040548900002D310110BA000080B582B013
:1041000000AF786039607B6800225A637B68114A8F
:104110001A637A683B685B78002B01D0002300E0CB
:104120000123101C01211A1CFFF72EFF3B68596860
:104130003B689A683B681B7B7868FFF755FF7A6895
:104140003B681B78101C00211A1CFFF71DFFBD46A1
:1041500002B080BDCFFF010080B588B000AF7860AD
:104160007B68BD4A934205D1BC4BBB61BB699B6870
:104170007B6101E0FC23EBE17B689B6A3B613A6970
:10418000C023DB00134014D03A6980239B00134006
:1041900003D0BB69FD225A7007E03A698023DB0037
:1041A000134002D0BB69FE225A70BB6909221A7003
:1041B000BAE1BB691B78082B00D9ADE19A00A84B86
:1041C000D3181B689F467B695B881A1C1023134019
:1041D0000AD07B691B881B0A9BB21A1C062313405A
:1041E000F0221343FB610FE07B691B881A1CFE233E
:1041F0001340FB617B695B881A1C0223134003D0C8
:10420000FB6901221343FB61BB6901221A707B68C1
:10421000FA695A627B6801225A6085E13B69802213
:1042200013400CD07B6880221A63BB69FF225A704E
:10423000BB6908221A707B6802225A6030E03B6931
:10424000402213402CD07B6840221A637B695B8834
:104250001A1C102313400AD0BB6902221A707B6912
:104260001B881A1CFF231A407B685A6218E07B697E
:104270005B881A1C022313400ED0BB6907221A70F8
:10428000BB691B797A69DB00D3181B89012B07D125
:104290007B6808225A6047E1BB6905221A7042E137
:1042A00042E13B69802213400CD07B6880221A6374
:1042B000BB69FF225A70BB6908221A707B68022210
:1042C0005A6014E03B694022134010D07B684022C2
:1042D0001A637B695B881A1C0223134003D0BB69F5
:1042E00003221A701FE1BB6905221A701BE11BE152
:1042F0007B695B881A1C102313400AD07B691B88DA
:104300001B0A9BB21A1C06231340F0221343FB61C5
:1043100005E07B691B881A1CFE231340FB617B6947
:104320005B881A1C0423134003D0FB69012213434A
:10433000FB61BB6904221A707B6801225A607B68AA
:10434000FA695A62F0E03B69802213400CD07B6826
:1043500080221A63BB69FF225A70BB6908221A7057
:104360007B6802225A6014E03B694022134010D05F
:104370007B6840221A637B695B881A1C0423134004
:1043800003D0BB6907221A7003E0BB6905221A70CB
:10439000C9E0C9E0BB695A88BB691B797969DB0050
:1043A000CB181B899A4224D3BB6900225A80BB696F
:1043B0001B790133DAB2BB691A717B695B881A1CFD
:1043C0000423134003D0BB6903221A70ABE07B695E
:1043D0005B881A1C0123134003D1BB691B79012B95
:1043E00006D9BB6908221A707B6802225A609BE0DA
:1043F00099E0BB691B797A69DB00D3185A68BB69FD
:104400005B88591C88B2B9694880D3181B781A1C7C
:104410007B685A62BB6906221A7085E03B6980227C
:1044200013400CD07B6880221A63BB69FF225A704C
:10443000BB6908221A707B6802225A600AE03B6955
:104440004022134006D07B6840221A63BB690522D4
:104450001A7068E068E0C04600A000401C0F002011
:1044600014BA00003B692022134046D0BB691B7977
:104470007A69DB00D3181B89FB607B68DA690B2340
:10448000FB181A70BB695B881A1EFB689A4210D22F
:10449000BB691B797A69DB00D3185A68BB695B88F2
:1044A000591C88B2B9694880D3180B22BA181278FF
:1044B0001A70BB695B881A1EFB689A420CD3FB68B2
:1044C000012B02D17B6808225A60BB6908221A704E
:1044D0007B6802225A6010E07B6804225A60FB6805
:1044E000012B0AD9BB695B881A1CFB68013B9A4205
:1044F00003D17B6808225A6016E015E03A698023F0
:104500005B00134007D07B68802252001A63BB69AE
:1045100009221A7008E007E0BB69FB225A70BB69E8
:1045200009221A7000E027E6BB691B78092B0BD122
:104530007B6800225A63BB695B785BB2012B05D1B3
:10454000BB6900225A7001E0012301E0BB695B787E
:104550005BB2181CBD4608B080BDC04680B584B0B3
:1045600000AF786039607B68294A934207D1294BB4
:10457000FB607B689B680122134005D001E0FC23AF
:1045800040E07B6820225A603B685B881A1C02234B
:10459000134003D03B681B89002B09D03B685B8824
:1045A0001A1C0423134005D03B681B8A002B01D141
:1045B000FC2327E0FB6800221A70FB6801225A7076
:1045C000FB6800225A80FB6800221A71FB683A6877
:1045D0009A607B68C0225A607B689B6A20221340E5
:1045E00001D07B68DB697B680B4A1A637B685B6B75
:1045F000FC22D2001A437B685A637B68181CFFF7C1
:10460000ABFD031C5BB2181CBD4604B080BDC046A8
:1046100000A000401C0F0020CFFF010080B582B039
:1046200000AF2A4B2A4ADA63284B284A92680121B4
:104630008A439A60FBF7B2FDE0231B03181CFEF7C8
:1046400043FE031C7B607B68224A93421CD97A6834
:10465000131C9B009B185B009B18181C0A2105F07B
:1046600021FF031C7B607B68181C1B4905F01AFFA7
:10467000031C01333B60154B144A126D174911405E
:104680003A680A431A651EE07A68131CDB009B1A1D
:10469000DB009B1A181C0A2105F004FF031C7B6039
:1046A0007B68181C0C4905F0FDFE031C01333B60C0
:1046B000064B064A126D094911403A680A438021A7
:1046C00049020A431A65BD4602B080BD00000C4095
:1046D000711B0000804F120040420F00C0FFFEFF20
:1046E00080B500AF054B054A926801218A439A6064
:1046F000024B0022DA63BD4680BDC04600000C407C
:1047000080B586B000AFF860B9607A60FB681B685E
:104710007B61BB6801229A40131CDB431A1C7B6936
:104720001A407B6801211940BB6899400B1C1A4351
:10473000FB681A60BD4606B080BDC04680B582B039
:1047400000AF78607B68044A944663449B0A181C57
:10475000BD4602B080BDC04600A0F7BF80B582B0A4
:1047600000AF786039607B68DB6A0122134000D0BB
:1047700005E0C0467B681B6B3A681340FAD1BD4622
:1047800002B080BD80B586B000AFF860B9607A60D5
:10479000FB681B687B617B69032213400AD0FB68BE
:1047A000181C0121FFF7DAFF7B69032293431A1CCF
:1047B000FB681A60FB68181C0421FFF7CFFFFB6839
:1047C000BA685A61FB68181C0621FFF7C7FFFB682F
:1047D00002225A60FB68181C0221FFF7BFFFFB682A
:1047E00001225A607A68BB689A420FD0FB68181C95
:1047F0000221FFF7B3FFFB687A685A61FB68181C57
:104800000621FFF7ABFFFB6802225A607B69032297
:10481000134007D0FB68181C0321FFF79FFFFB68BC
:104820007A691A60BD4606B080BDC04680B582B0C8
:1048300000AF7860081C111CFB1C021C1A70BB1C0A
:104840000A1C1A70FB1C1B78002B02D0012B0BD00A
:1048500015E07B683C331A1CBB1C1B78101C042120
:104860001A1CFFF74DFF0AE07B683C331A1CBB1C87
:104870001B78101C0A211A1CFFF742FFC046BD46D8
:1048800002B080BD80B586B000AF786039607B68CB
:10489000181CFFF753FF031CFB607B68DB6B634A4C
:1048A00013407B613B68DB7C1A1C3B681B7D9B01D2
:1048B00013437A6913437B617B687A69DA63002367
:1048C0007B613B681B7B002B03D07B690822134371
:1048D0007B613B685B7B002B03D07B690422134325
:1048E0007B613B689B7B002B03D07B6910221343C9
:1048F0007B613B68DB7B002B04D07B69802252000C
:1049000013437B613B681B7C002B04D07B698022B6
:10491000920013437B613B685B7C9B021A1C7B69A2
:1049200013437B6100233B613B689B7C022B04DCCF
:10493000012B0BDA002B03D00CE0032B03D009E092
:1049400003233B6106E000233B6103E03B689B7C63
:104950003B61C0463B699B037A6913437B617B687B
:10496000181C05210122FFF7CBFEFB68181C002153
:10497000FFF726F83B681B78023B012B22D83B68E7
:104980001B781A1C7B6913437B617B68181C01210F
:10499000FFF7E4FE7B6820221A607B68181C012167
:1049A000FFF7DCFEFB68181C0121FFF709F83B68E4
:1049B0009A687B685A617B6802225A607B687A69D0
:1049C0001A602FE07B681B680322134009D07B69C3
:1049D00020221A437B681A607B68181C0121FFF7AC
:1049E000BDFE7B68181C05210022FFF789FE3B688D
:1049F0005A683B689B687968081C111C1A1CFFF7F1
:104A0000C1FE3B681B78012B0BD17B68181C012170
:104A1000FFF7A4FE3B681B781A1C7B691A437B686E
:104A20001A60C046BD4606B080BDC04638FEFFFFD6
:104A300080B584B000AFF860B9607A603B60094926
:104A4000BA68FC239B031A407B68072003401A4383
:104A50003B681A43FB6804339B005A50BD4604B0C0
:104A600080BDC04600C00C4080B584B000AFF86087
:104A7000B9607A600949BA68FC239B031A407B68D5
:104A8000072003401343802252051A43FB68043376
:104A90009B005A50BD4604B080BDC04600C00C40CB
:104AA00080B586B000AFF860B9607A60FB681B68BB
:104AB0007B61BB6801229A40131CDB431A1C7B6993
:104AC0001A407B6801211940BB6899400B1C1A43AE
:104AD000FB681A60BD4606B080BDC04680B584B094
:104AE00000AF78607B68002B02D0012B04D007E078
:104AF000074B9B68FB6006E0054BDB68FB6002E050
:104B00000023FB60C046FB68181CBD4604B080BD96
:104B10000000084080B584B000AF786039607B68E1
:104B2000012B04D83B681B0E1B0600D1C0467B68D6
:104B3000002B02D0012B03D008E0064BFB6002E003
:104B4000054BFB60C046FB683A681A60BD4604B07E
:104B500080BDC046080008400C00084080B582B007
:104B600000AF021CFB1D1A70FB1D1B78044A101CB1
:104B700000211A1CFFF794FFBD4602B080BDC0465D
:104B80000000084080B582B000AF021CFB1D1A7007
:104B9000FB1D1B78002B03D0044B01221A6202E09C
:104BA000024B00221A62BD4602B080BD00000840E0
:104BB00080B584B000AF78607B681B78002B02D092
:104BC0000123FB6001E00023FB607B685B78002B26
:104BD00003D0FB6802221343FB607B689B78002BA9
:104BE00003D0FB6804221343FB60034BFA681A608E
:104BF000BD4604B080BDC0460000084080B500AF8F
:104C00000020FFF7ABFF0120FFF7A8FFBD4680BDE6
:104C100080B582B000AF786039607B68384A9342D3
:104C200007D07B68374A934203D07B68364A934269
:104C300000D1C0463B681B7801225340DBB2002BF9
:104C400002D07B6802225A607B6800225A623B686D
:104C50009B781A063B68DB781B041A433B689B79F8
:104C60009B021A433B68DB791B0213433A68127AB2
:104C70001A433B685B78002B01D0402300E00023FF
:104C80001A433B685B7A002B01D0802300E00023AD
:104C90001A433B689B7A002B01D0202300E00023BD
:104CA0001A433B68DB7A002B01D0102300E000237D
:104CB0001A433B681B79002B02D080239B0100E044
:104CC00000231A433B685B79002B02D080235B05ED
:104CD00000E000231A433B681B7B002B01D0082314
:104CE00000E000231A437B681A603B681B78002BA6
:104CF00002D07B6801225A60BD4602B080BDC0462A
:104D000000000140000401400008014080B584B06B
:104D100000AFF860B9607A60FB68284A934207D018
:104D2000FB68274A934203D0FB68264A934200D18E
:104D3000C0467B681B789A067B685B781B061A4323
:104D40007B689B781B041A437B68DB781B031A4340
:104D50007B681B799B021A437B685B791B021343B8
:104D60007A6892791A437B68DB79002B02D0802322
:104D70009B0300E000231A437B681B7A002B02D0C0
:104D800080235B0300E000231A437B685B7A002BDF
:104D900001D0102300E000231A437B689B7A002B8C
:104DA00001D0042300E000231A43111CFB68BA68F9
:104DB00003321201D150BD4604B080BD0000014055
:104DC000000401400008014080B584B000AFF860E5
:104DD000B9607A60FB681B68BA68D2431A407B6886
:104DE0001A43FB681A60BD4604B080BD80B586B02A
:104DF00000AFF860B9607A60BB68002B05D1184B32
:104E0000181CFEF761FA031CBB60BB685B007B618A
:104E10007A687B69D318013B7B617869796805F012
:104E200041FB031C7B617B69043B7B617B699B01CC
:104E30007B617B69C0337B617B69FF2293437B612C
:104E40007B69084A13407B61FB6814331A1C0549CF
:104E50007B69101C1A1CFFF7B7FFBD4606B080BD6A
:104E600040810400C0FF1F0080B582B000AF7860B1
:104E700039607B682C4A934203D07B682B4A93426B
:104E800000D1C0467B68181C00F052F87B681A6895
:104E90003B681B8A01210B439BB2191C3B689B7B1F
:104EA000002B02D08023DB0000E000230B431A43D9
:104EB0007B681A607B681A683B681B7D002B02D0F8
:104EC00080239B0500E000231A437B681A603B683F
:104ED0009B7C002B07D03B68DB7C10221343DBB2AA
:104EE0001A1C7B689A653B681B7B1A1C80235B013C
:104EF0001A437B685A603B685A683B689B687968CC
:104F0000081C111C1A1CFFF771FF3B685B7B002B10
:104F100002D07B681022DA603B681B781A1C7B6821
:104F2000DA60BD4602B080BD00C0004000C4004051
:104F300080B582B000AF78607B681E4A934203D090
:104F40007B681D4A934200D1C0467B681B4ADA60E9
:104F50007B6800221A607B68194A5A607B680022CD
:104F60009A607B6800225A617B680022DA647B6861
:104F7000144A9A647B6800225A657B680D4A934202
:104F800003D07B680C4A934202D17B6800221A65E9
:104F90007B6800229A657B68064A934203D07B684F
:104FA000054A934202D17B680022DA65BD4602B011
:104FB00080BDC04600C0004000C40040AA0E0000F2
:104FC00005100000F91F000080B582B000AF7860C6
:104FD0000A1CFB1C1A70C0467B681B6940221340E8
:104FE000FAD0FB1C1A787B685A63BD4602B080BDBC
:104FF00080B582B000AF78600A1CBB1C1A80C04626
:105000007B681B6940221340FAD0BB1C1A887B685E
:10501000DA63BD4602B080BD80B582B000AF786073
:1050200039607B681A683B68DA40131C0122134020
:10503000181CBD4602B080BD80B500AF044B044AC9
:10504000126904218A431A6130BFBD4680BDC04643
:1050500000ED00E080B582B000AF021C3960FB1D9E
:105060001A70FB1D1B78002B0DD0FB1D1B78012B2C
:1050700009D0FB1D1B78022B05D0FB1D1B78032BD1
:1050800001D0FB1D1B78FB1D1A78131CDB009B183D
:105090009B001C33054A9A183B68101C191CFFF72B
:1050A000BBFF031C181CBD4602B080BD0060004061
:1050B00090B585B002AF041C3960101C191CFB1D93
:1050C000221C1A70BB1D021C1A707B1D0A1C1A7050
:1050D000FB1D187839683A68BB1D1C787B1D1B784E
:1050E00000931823FB181B780193231CFEF71AFE6C
:1050F000BD4603B090BDC04680B582B000AF7860B9
:105100007B68DB68181CBD4602B080BD80B582B0EC
:1051100000AF786039607B683A681A62BD4602B0B9
:1051200080BDC04680B582B000AF78607B689B6967
:10513000181CBD4602B080BD80B582B000AF78605B
:105140003960074B064A52683968C94311407A688A
:10515000386802400A435A60BD4602B080BDC0466E
:1051600000C00C4080B582B000AF7860034B7A6815
:105170003F210A401A60BD4602B080BD00C00C400D
:1051800080B582B000AF78607B685B6A181CBD4652
:1051900002B080BD80B582B000AF78600A1CFB1CF5
:1051A0001A707B680C4A934207D07B680B4A934283
:1051B00003D07B680A4A934200D1C046FB1C1B788F
:1051C000002B03D07B6801225A6002E07B68022238
:1051D0005A60BD4602B080BD00000140000401409D
:1051E0000008014080B582B000AF0A4B181C622154
:1051F00004F00CFB031C7B60064B181C642104F0BC
:1052000005FB021C7B6813437B607B68181CBD4652
:1052100002B080BD00A0004080B582B000AF0B4B53
:10522000181C6221002204F0B5FA031C7B60074BB6
:10523000181C6421002204F0ADFA021C7B681343A1
:105240007B607B68181CBD4602B080BD00A000409A
:1052500080B588B002AF2E4B1B78DBB201225340E1
:10526000DBB2002B04D005F0F5F8294B01221A70AF
:10527000284B1B78DBB2002B04D000F09FFE254B9F
:1052800000221A70244ABB1D0093101C62210022C8
:10529000002304F059F9031CBB601F4A3B1D009317
:1052A000101C64210022002304F04EF9021CBB688C
:1052B0001343BB60BB68002B1DD1BB1D1B881BB2F9
:1052C0000020191C04F030FA031C7B613B1D1B8875
:1052D0001BB20020191C04F027FA031C3B61BB1D04
:1052E0001A883B1D1B8812B21BB2101C191C00F03F
:1052F00015F8031CFB60BB685A1E9341D8B279694C
:105300003A69FB6801F0A0FABD4606B080BDC04610
:10531000740F0020720F002000A0004090B58DB0E7
:1053200000AF021CBB1D1A803B1D0A1C1A80012302
:105330005B42BB62BB1D00229B5E181C05F082FC19
:10534000041C3B1D00229B5E181C05F07BFC031C0B
:105350009C4225DABB1D00229B5EFA2292005A4332
:105360003B1D00215B5E101C191C05F02BF9031C72
:105370007B623B1D00229B5E002B08DD2F23FB1868
:105380001A221A702E23FB1824221A702DE02F23C4
:10539000FB1808221A702E23FB1812221A7024E020
:1053A0003B1D00229B5EFA2292005A43BB1D002146
:1053B0005B5E101C191C05F005F9031C7B62BB1D0C
:1053C00000229B5E002B08DD2F23FB1811221A7090
:1053D0002E23FB181B221A7007E02F23FB18FF2235
:1053E0001A702E23FB1809221A702D23FB182F2266
:1053F000BA1812781A70C6E02D23FB181B785BB21E
:1054000001330CD10020232100F04CFE031CBB61B2
:105410000120232100F046FE031C7B6113E02D23B5
:10542000FB181B785BB20020191C00F03BFE031C2C
:10543000BB612D23FB181B785BB20120191C00F007
:1054400031FE031C7B612D23FB181B785BB2232BE1
:105450000CD10020002100F025FE031C3B6101203F
:10546000002100F01FFE031CFB6015E02D23FB183C
:105470001B785BB201330020191C00F013FE031CE3
:105480003B612D23FB181B785BB201330120191CF3
:1054900000F008FE031CFB602F23FB181B785BB297
:1054A0001A2B05D02F23FB181B785BB2082B14D1C5
:1054B000BB69FA2292005343181C796905F082F8FF
:1054C000031C3B623B69FA2292005343181CF968A3
:1054D00005F078F8031CFB6113E07B69FA22920067
:1054E0005343181CB96905F06DF8031C3B62FB6857
:1054F000FA2292005343181C396905F063F8031C23
:10550000FB617A6A3B6A9A4203DB7A6AFB699A42D8
:1055100007DD7A6A3B6A9A422CDC7A6AFB699A4216
:1055200028DB2D23FB1800229A56131C9B009B1886
:105530005B001C1C7A6A3B6AD11A2D23FB181B786E
:105540005BB25A1C131C9B009B185B00181C2D237C
:10555000FB181B785BB20A2252425343C3185943CB
:10556000FA693B6AD31A081C191C05F02BF8031CB6
:10557000E318BB622D23FB181B78DBB20133DAB2D0
:105580002D23FB181A702D23FA182E23FB181278DE
:1055900052B21B785BB29A4200DA2DE7BB6A002B4D
:1055A00001DBBB6A3AE1BB1D00229B5E181C05F0C3
:1055B00049FB041C3B1D00229B5E181C05F042FBAE
:1055C000031C9C4225DBBB1D00229B5EFA2292003D
:1055D0005A433B1D00215B5E101C191C04F0F2FFB6
:1055E000031C7B623B1D00229B5E002B08DD2F23EA
:1055F000FB181A221A702E23FB1824221A702DE091
:105600002F23FB1808221A702E23FB1812221A705F
:1056100024E03B1D00229B5EFA2292005A43BB1DF0
:1056200000215B5E101C191C04F0CCFF031C7B6284
:10563000BB1D00229B5E002B08DD2F23FB181122CF
:105640001A702E23FB181B221A7007E02F23FB1859
:10565000FF221A702E23FB1809221A702D23FB1823
:105660002F22BA1812781A70C6E02D23FB181B7867
:105670005BB201330CD10020232100F013FD031C89
:10568000BB610120232100F00DFD031C7B6113E0B1
:105690002D23FB181B785BB20020191C00F002FDC3
:1056A000031CBB612D23FB181B785BB20120191C66
:1056B00000F0F8FC031C7B612D23FB181B785BB208
:1056C000232B0CD10020002100F0ECFC031C3B61DB
:1056D0000120002100F0E6FC031CFB6015E02D23F7
:1056E000FB181B785BB201330020191C00F0DAFCB8
:1056F000031C3B612D23FB181B785BB20133012097
:10570000191C00F0CFFC031CFB602F23FB181B7837
:105710005BB21A2B05D02F23FB181B785BB2082B2A
:1057200014D1BB69FA2292005343181C796904F022
:1057300049FF031C3B623B69FA2292005343181C49
:10574000F96804F03FFF031CFB6113E07B69FA2258
:1057500092005343181CB96904F034FF031C3B62E8
:10576000FB68FA2292005343181C396904F02AFF9F
:10577000031CFB617A6A3B6A9A4203DC7A6AFB6922
:105780009A4207DA7A6A3B6A9A422CDB7A6AFB69A8
:105790009A4228DC2D23FB1800229A56131C9B00EA
:1057A0009B185B001C1C7A6A3B6AD11A2D23FB18DC
:1057B0001B785BB25A1C131C9B009B185B00181CC7
:1057C0002D23FB181B785BB20A2252425343C318A5
:1057D0005943FA693B6AD31A081C191C04F0F2FEFB
:1057E000031CE318BB622D23FB181B78DBB20133CB
:1057F000DAB22D23FB181A702D23FA182E23FB186A
:10580000127852B21B785BB29A4200DA2DE7BB6A7B
:10581000002B01DBBB6A01E00A235B42181CBD467A
:105820000DB090BD80B582B000AFBB1D00221A70D4
:1058300002200021FFF70EFC021CBB1D1A70022083
:105840000121FFF707FC021C7B1D1A70BB1D1B7892
:10585000002B06D17B1D1B78012B02D1FB1D0122E1
:105860001A70BB1D1B78012B06D17B1D1B78012BE9
:1058700002D1FB1D02221A70BB1D1B78012B06D121
:105880007B1D1B78002B02D1FB1D03221A70BB1D50
:105890001B78002B06D17B1D1B78002B02D1FB1D32
:1058A00004221A70FB1D1B78181CBD4602B080BD77
:1058B00080B500AF064B181CFFF71EFC031CDBB2C3
:1058C0000F3BDBB2DBB25BB2181CBD4680BDC046ED
:1058D0000060084080B582B000AFBB1D02221A7084
:1058E0007B1D03221A70FB1D00221A700CE07B1D29
:1058F0001B7801229A40131C181CFFF733FCFB1D78
:105900001A78FB1D01321A70FB1D1B78032BEED990
:105910004BE0BB1D1B7801229A407B1D1B780121A7
:1059200099400B1C13430020191CFFF705FC7B1D3D
:105930001B7801229A40131C181CBB1D1B780122E6
:105940009A407B1D1B78012199400B1C1343191CA5
:10595000FFF7F2FB7B1D1B7801229A40BB1D1B78D1
:10596000012199400B1C1343181CBB1D1B780122FD
:105970009A407B1D1B78012199400B1C1343191C75
:10598000FFF7DAFBBB1D1B7801229A40131C181C81
:10599000BB1D1B7801229A407B1D1B780121994079
:1059A0000B1C1343191CFFF7C7FBFFF781FF031EF6
:1059B000AFD1BD4602B080BD90B587B000AF1A4BE5
:1059C000181C0121FDF726FC184B181C0121FDF7BE
:1059D00021FC3B1C164A13CA13C313CA13C3154B2D
:1059E000181C00210122FEF721FF124B181C012177
:1059F0000122FEF71BFF0F4A3B1C101C191CFEF76F
:105A000041FFFFF767FFC0239B030220191C002200
:105A1000FFF72AF8C0239B030320191C0122FFF77C
:105A200023F8BD4607B090BD000A1A0000620400CA
:105A300038BA00000060084080B582B002AF002391
:105A400000930220002101220123FFF731FB0023F4
:105A500000930220012101220023FFF729FBBD460C
:105A600080BDC04680B500AF064B181C0021FDF775
:105A7000D1FB054B181C0021FDF7CCFBFFF7DCFF29
:105A8000BD4680BD000A1A000062040080B582B0E5
:105A900000AF074B181CFFF745FB031C7B60044A53
:105AA0007B68101C191CFFF731FBBD4602B080BD9E
:105AB0000060084080B582B002AF0A4B01221A7024
:105AC000012300930220002101220123FFF7F0FAB5
:105AD000012300930220012101220123FFF7E8FAAC
:105AE000BD4680BD2C0F002080B582B002AF0A4BAE
:105AF00000221A70002300930220002101220123BA
:105B0000FFF7D6FA0123009302200121012200238E
:105B1000FFF7CEFABD4680BD2C0F002080B500AF48
:105B2000084B1B7801225340DBB2002B02D0FFF759
:105B3000C1FF05E0034B1B78002B01D0FFF7D4FF1A
:105B4000BD4680BD2C0F002080B582B000AFFFF7AE
:105B500049FB031C7B60FFF7C7FFFFF72DFF7B6846
:105B6000181CBD4602B080BD90B585B000AF0023C3
:105B7000BB600F23FB1800221A701F4B1B78DBB28F
:105B800001225340DBB2002B06D0FFF7DDFF031CE0
:105B9000BB60194B01221A70184B1B78DBB2002B2B
:105BA00004D0FFF7BBFF154B00221A70144B1B7873
:105BB000002B05D00F23FC18FFF734FE031C2370C5
:105BC000FC1DFFF775FE031C2370FFF70BFB031C86
:105BD000BB60BB685A1E9341D9B2FB1D00229A5686
:105BE0000F23FB181B78081C111C1A1C00F028FF3F
:105BF000BD4605B090BDC046740F0020710F002057
:105C00002C0F002080B588B000AF11200521FDF7D2
:105C1000E9FC0320FDF706FE2B4B181C0121FDF7C4
:105C2000F9FA2A4B181C0121FDF7F4FAC0239B0353
:105C30000220191C00220023FEF7FAFEC0239B035A
:105C40000320191C01220023FEF7F2FE1423FA1888
:105C50001F4B111C1A1C0B23081C111C1A1C05F0CD
:105C600031F81C4A1423FB18101C00211A1CFFF7E2
:105C70004DF81423FB1802229A70164A1423FB18BD
:105C8000101C01211A1CFFF741F83B1D00221A606D
:105C900000225A6000229A6000221A733B1D0122E2
:105CA0001A703B1D01225A703B1D03221A723B1DC4
:105CB00001229A72074A3B1D101C191CFEF7A8FF0F
:105CC000BD4608B080BDC04600620400000204006A
:105CD00050BA00000000014080B500AF024B052221
:105CE0005A62BD4680BDC0460000014080B582B00A
:105CF00000AFFFF777FA031C7B6004F09DFBFFF712
:105D000081FFFFF7E9FFFFF7D5FE7B68181CBD4652
:105D100002B080BD80B582B000AF094B181CFFF700
:105D20002FFA031C7B60FFF7D7FF7B68042B01D899
:105D3000012300E00023181CBD4602B080BDC04610
:105D40000000014080B584B000AF021CFB1D1A703A
:105D5000FFF7E0FF031E0FD0FB1D1B78012B04D1C2
:105D60000F23FB1808221A7015E00F23FB18FA1DE9
:105D70001278013A1A700EE0FB1D1B78082B04D133
:105D80000F23FB1801221A7005E00F23FB18FA1DE0
:105D9000127801321A700F23FB181B78181CBD46AD
:105DA00004B080BD80B500AFFFF746F9BD4680BDA9
:105DB00080B500AF0B4B181C0021FFF7EBF90A4B25
:105DC000181C0021FDF726FA084B181C0021FDF7CE
:105DD00021FAFFF731FEFFF71FFA054B00221A7078
:105DE000BD4680BD000001400002040000620400C6
:105DF000740F002090B583B000AFFB1D01221A7014
:105E0000FFF774FF43E0264B1B78DBB2002B09D071
:105E1000244BFA1D12781A70FFF7CAFF204B00229C
:105E20001A7039E0204B1B78DBB2002B04D11F4BDA
:105E30001B78DBB2002B11D0BC1DFB1D1B78181C7E
:105E4000FFF780FF031C2370FB1DBA1D12781A7028
:105E5000154B00221A70154B00221A70FFF7C2F979
:105E6000031C3B603B685A1E9341DAB2FB1D1B7852
:105E7000101C191C00F0DAF90B4B1B78DBB21A1C52
:105E80000A4B1B78DBB2134301D1FFF78BFF054BA5
:105E90001B78DBB2002BB6D0BD4603B090BDC04628
:105EA000700F00206F0F0020710F0020730F002073
:105EB00080B500AF72B6074B1B68013304D0054BA9
:105EC0001B685A1C034B1A60024B1B68181CBD460A
:105ED00080BDC046280F002080B582B000AF0B4BBC
:105EE0001B68002B0DD0094B1B685A1E074B1A600C
:105EF000064B1B687B607B68002B00D162B67B6819
:105F000000E00023181CBD4602B080BD280F002011
:105F100080B500AF02E00120FDF742FE064B1B7882
:105F2000DBB201225340DBB2002BF4D1024B002242
:105F30001A70BD4680BDC046710F002080B582B08A
:105F400000AFFE231B057B60FFF7B2FFFEF766FB89
:105F50007B68181C05F0ECFAFEF7C2FBFFF7BCFFEC
:105F6000BD4602B080BDC04680B586B000AFF860C7
:105F7000B9607A60FE231B057B61BA68131CDB00E5
:105F80009B189B001A1C7B68D3189B007A69D31856
:105F90007B61FB683B61FFF78BFFFEF73FFB7A6994
:105FA0001023FB18101C191C042205F0C9FAFEF777
:105FB00097FBFFF791FFBD4606B080BD90B58BB053
:105FC00002AF0023BB613B1C00221A7004F034FABC
:105FD000304B00221A700023FB614AE0FA69131C5F
:105FE0009B009B185B001C1C3A1C2B4B101C191CA3
:105FF000221C04F079FE3B1C181C01F003FDFFF786
:1060000087FFFB69002B01D1FFF798FF234A162376
:10601000FB180093101C62210022002303F094FA65
:10602000021CBB691343BB611C4A1423FB18009379
:10603000101C64210022002303F086FA021CBB69B5
:106040001343BB611623FB181B881AB2FB69101C93
:1060500000211A1CFFF788FF1423FB181B881AB2B3
:10606000FB69101C01211A1CFFF77EFFFB6901333D
:10607000FB61FB69232BB1DDBB69002B05D1084B0C
:10608000181C01212422FFF76FFF04F0E3F9BD463D
:1060900009B090BD710F0020ECBA000000A00040D4
:1060A000CC07000080B584B000AF78603960FE2373
:1060B0001B05FB60FB682133FF331B68104A9342CA
:1060C0000DD17A68131CDB009B189B001A1C3B68DF
:1060D000D3189B00FA68D3181B689BB20AE07A6851
:1060E000131CDB009B189B001A1C3B68D218054B45
:1060F0005200D35A1BB2181CBD4604B080BDC04626
:10610000CC0700005CBA000080B500AF064A074B20
:10611000101C191CFCF7CEFB034B00225A60024BEB
:10612000034A9A60BD4680BD300F0020ACB8000025
:10613000FFFFFF0080B582B000AFFAF7F1F8031C53
:106140007B607B68002B00D0FEE70020FBF7F6FCAD
:10615000031C7B607B68002B00D0FEE7074B181CFC
:10616000FCF72AF8031C7B607B68002B00D0FEE75D
:10617000FFF7CAFFBD4602B080BDC046300F002009
:1061800090B583B002AF254B1B681B885B089BB2A0
:106190001C3B1C1C214B1B685B885B089BB21E3B95
:1061A0001E491F4A009300230193081C111C0F2253
:1061B000231CFCF717FB194B1B681B885B089BB261
:1061C000283B1C1C154B1B685B885B089BB20F3B74
:1061D0001249144A009300230193081C111C0F223A
:1061E000231CFCF7FFFA0D4B1B681B885B089BB256
:1061F000323B1C1C094B1B685B885B089BB2053358
:106200000649094A009300230193081C111C0F2220
:10621000231CFCF7E7FABD4601B090BD300F00200B
:10622000F8BA000000BB00000CBB000090B589B0BC
:1062300002AF021CFB1D1A70BB1D0A1C1A70A44B76
:10624000181CFCF785F8FB1D1B78002B02D0FFF70C
:1062500097FF37E19E4B1B681B885B089BB2243B72
:106260001C1C9B4B1B685B885B089BB23C3B9849A2
:10627000984A009300230193081C111C0F22231C31
:10628000FCF7B0FA924B1B681B885B089BB2343B4F
:106290001C1C8F4B1B685B885B089BB22D3B8C4999
:1062A0008D4A009300230193081C111C0F22231C0C
:1062B000FCF798FA864B1B681B885B089BB2343B43
:1062C0001C1C834B1B685B885B089BB2233B80498B
:1062D000824A009300230193081C111C0F22231CE7
:1062E000FCF780FA0823FA187D4B101C191C04F0E7
:1062F000FBFCBB1D1B781A1C9200D318DB18DBB209
:106300001E3BDAB21723FB181A70714B1B681B88EF
:106310005B089BB23C3B1C1C6D4B1B685B885B089D
:106320009BB21A1C1723FB181B785BB2D318684961
:106330000822BA18009300230193081C111C0F2295
:10634000231CFCF74FFA624B1B681B885B089BB24F
:10635000383B1C1C5E4B1B685B885B089BB2143B84
:106360005B49604A009300230193081C111C0F2213
:10637000231CFCF737FA564B1B681B885B089BB243
:10638000383B1C1C524B1B685B885B089BB20A3B6A
:106390004F49554A009300230193081C111C0F22FA
:1063A000231CFCF71FFA4A4B1B681B885B089BB237
:1063B000383B1C1C464B1B685B885B089BB24449FE
:1063C0004A4A009300230193081C111C0F22231C2E
:1063D000FCF708FA3E4B1B681B885B089BB2383BF6
:1063E0001C1C3B4B1B685B885B089BB20A3338491B
:1063F0003F4A009300230193081C111C0F22231C09
:10640000FCF7F0F9324B1B681B885B089BB2383BEA
:106410001C1C2F4B1B685B885B089BB214332C49F8
:10642000344A009300230193081C111C0F22231CE3
:10643000FCF7D8F9264B1B681B885B089BB2383BDE
:106440001C1C234B1B685B885B089BB21E332049D6
:10645000294A009300230193081C111C0F22231CBE
:10646000FCF7C0F91A4B1B681B885B089BB2383BD2
:106470001C1C174B1B685B885B089BB228331449B4
:106480001E4A009300230193081C111C0F22231C99
:10649000FCF7A8F90E4B1B681B885B089BB2383BC6
:1064A0001C1C0B4B1B685B885B089BB23233084992
:1064B000134A009300230193081C111C0F22231C74
:1064C000FCF790F9FBF7D2FDBD4607B090BDC04682
:1064D000300F002018BB000024BB000034BB0000BC
:1064E00044BB000048BB000054BB000064BB00007C
:1064F00074BB000084BB000094BB0000A0BB000084
:10650000ACBB0000B0B58AB002AFF860B9607A6089
:10651000FB68181CFA23990004F054F8031C181C9B
:1065200004F090FB051CFB68181CFA23990004F08A
:106530002FF90B1C181C04F085FB031C181C64218C
:1065400004F040F8031C1C1C1023FA18474B101CC5
:10655000191C2A1C231C04F0C7FBFB68002B03DA60
:106560001023FB182D221A71414B1B681B885B08F6
:106570009BB22A3B1C1C3E4B1B685B885B089BB292
:106580000A3B3B491022BA18009300230193081CD0
:10659000111C0F22231CFCF725F9BB68181CFA23D9
:1065A000990004F00FF8031C181C04F04BFB051CA9
:1065B000BB68181CFA23990004F0EAF80B1C181C9D
:1065C00004F040FB031C181C642103F0FBFF031CB8
:1065D0001C1C1023FA18274B101C191C2A1C231CE6
:1065E00004F082FBBB68002B03DA1023FB182D227A
:1065F0001A711F4B1B681B885B089BB22A3B1C1C33
:106600001B4B1B685B885B089BB219491022BA18A8
:10661000009300230193081C111C0F22231CFCF77C
:10662000E1F81023F918144A7B68081C111C1A1C85
:1066300004F05AFB0E4B1B681B885B089BB2283B7F
:106640001C1C0B4B1B685B885B089BB20A33084918
:106650001022BA18009300230193081C111C0A226F
:10666000231CFCF7BFF8BD4608B0B0BDB8BB0000A6
:10667000300F0020C8BB0000D8BB000080B586B03A
:1066800000AF78607B68181C0F2103F09BFF031C90
:10669000FB607B68181C0F2104F07AF80B1CBB60B0
:1066A000FB68002B1BD1664B1B681B885B089BB2E9
:1066B000191C644ABB68D3181B785BB2CB187B618A
:1066C0005F4B1B685B885B089BB2191CBB680F2281
:1066D000D31A5C4AD35C5BB2CB1A3B6158E0FB68CF
:1066E000012B1BD1564B1B681B885B089BB2191CE6
:1066F000BB680F22D31A534AD35C5BB2CB187B61C1
:106700004F4B1B685B885B089BB2191C4D4ABB68EA
:10671000D3181B785BB2CB183B6139E0FB68022BC6
:106720001BD1474B1B681B885B089BB2191C454A51
:10673000BB68D3181B785BB2CB1A7B61404B1B68DC
:106740005B885B089BB2191CBB680F22D31A3D4AB9
:10675000D35C5BB2CB183B611AE0394B1B681B88DA
:106760005B089BB2191CBB680F22D31A354AD35C55
:106770005BB2CB1A7B61324B1B685B885B089BB2B8
:10678000191C304ABB68D3181B785BB2CB1A3B612B
:106790002B497A693B69081C111C1A1CFBF740FE47
:1067A0007B695A1C26493B69081C111C1A1CFBF703
:1067B00037FE7B695A1E22493B69081C111C1A1CB2
:1067C000FBF72EFE3B6901331D497A69081C111C39
:1067D0001A1CFBF725FE3B69013B19497A69081C25
:1067E000111C1A1CFBF71CFE7B695A1C3B69013308
:1067F0001349081C111C1A1CFBF712FE7B695A1E58
:106800003B69013B0E49081C111C1A1CFBF708FED2
:106810007B695A1E3B6901330949081C111C1A1C6B
:10682000FBF7FEFD7B695A1C3B69013B0449081CD0
:10683000111C1A1CFBF7F4FDBD4606B080BDC04616
:10684000300F0020FCBD000090B587B000AFB960EC
:106850007A603B600F23FB18021C1A70344B181C23
:10686000FBF776FD0F23FB181B78002B02D0FFF7F8
:1068700087FC57E0B9687A683B68081C111C1A1C31
:10688000FFF740FE1723FB180F221A7015E017239D
:10689000FB181B785BB23B2B06DC1723FB181B781D
:1068A0005BB2181CFFF7EAFE1723FB181B78DBB25C
:1068B0000133DAB21723FB181A701723FB180024D0
:1068C0001C573B68181C062103F07CFE031C0F3389
:1068D0009C42DCDD3A6887235B009A4222DD172365
:1068E000FB1800221A700FE01723FB181B785BB20D
:1068F000181CFFF7C3FE1723FB181B78DBB201330C
:10690000DAB21723FB181A701723FB1800241C5740
:106910003B680F3BFF3B181C062103F053FE031C92
:106920009C42E1DDFBF7A2FBBD4607B090BDC0462F
:10693000300F002080B582B000AF021CFB1D1A7022
:10694000BB1D0A1C1A70FB1D00229A56BB1D1B782A
:106950005BB23A49081C111C1A1CFBF761FDFB1DB8
:106960001B785BB25A1CBB1D1B785BB23349081CF9
:10697000111C1A1CFBF754FDFB1D1B785BB25A1E41
:10698000BB1D1B785BB22D49081C111C1A1CFBF7A0
:1069900047FDFB1D00229A56BB1D1B785BB20133DD
:1069A0002649081C111C1A1CFBF73AFDFB1D00228E
:1069B0009A56BB1D1B785BB2013B2049081C111C79
:1069C0001A1CFBF72DFDFB1D1B785BB25A1CBB1D6F
:1069D0001B785BB201331949081C111C1A1CFBF708
:1069E0001FFDFB1D1B785BB25A1EBB1D1B785BB2E3
:1069F000013B1249081C111C1A1CFBF711FDFB1D61
:106A00001B785BB25A1EBB1D1B785BB201330B496E
:106A1000081C111C1A1CFBF703FDFB1D1B785BB245
:106A20005A1CBB1D1B785BB2013B0449081C111C9E
:106A30001A1CFBF7F5FCBD4602B080BD300F0020EC
:106A400090B58BB002AF041C081C111CFB1D221C4E
:106A50001A70BB1D021C1A707B1D0A1C1A70A84BF1
:106A6000181CFBF775FCFB1D1B78002B02D0FFF7F1
:106A700087FBBFE10C23FA18A24B101C191C04F071
:106A800033F99F4B1B681B885B089BB2283B1C1C7F
:106A90009B4B1B685B885B089BB20C3B98490C22A4
:106AA000BA18009300230193081C111C0F22231C09
:106AB000FBF798FEBB1D1B785BB2181C04F0C2F8F4
:106AC000041C0C23FA18904B101C191C221C04F0F7
:106AD0000BF9BB1D1B787F2B03D90C23FB182D2230
:106AE0009A71874B1B681B885B089BB2233B1C1C5D
:106AF000834B1B685B885B089BB281490C22BA18E8
:106B0000009300230193081C111C0F22231CFBF788
:106B100069FE7B1D1B78002B00D16BE17B1D1B7870
:106B20000C22B918794A081C111C1A1C04F0DCF854
:106B3000734B1B681B885B089BB21E3B1C1C704B75
:106B40001B685B885B089BB214336D490C22BA1832
:106B5000009300230193081C111C0F22231CFBF738
:106B600041FE1F23FB1800221A703CE17B1D1B789D
:106B7000012B3ED1624B1B681B885B089BB2DAB2CB
:106B80001F23FB181B785BB20F21CB1A6049CB5C2B
:106B9000DBB2D318DAB21C23FB181A701E23FB18C1
:106BA0001C22BA1812781A70554B1B685B885B0858
:106BB0009BB2DAB21F23FB181B785BB25449CB5C43
:106BC000DBB2D318DAB21D23FB181A704C4B1B68CA
:106BD0005B885B089BB2DAB21F23FB181B785BB2A1
:106BE0004B49CB5CDBB2D31ADAB21B23FB181A7009
:106BF000D2E07B1D1B78022B3ED1414B1B681B88CA
:106C00005B089BB2DAB21F23FB181B785BB24049CA
:106C1000CB5CDBB2D318DAB21E23FB181A70384BE8
:106C20001B681B885B089BB2DAB21F23FB181B781A
:106C30005BB23749CB5CDBB2D31ADAB21C23FB1848
:106C40001A702F4B1B685B885B089BB2DAB21F235C
:106C5000FB181B785BB20F21CB1A2D49CB5CDBB242
:106C6000D318DAB21B23FB181A701D23FB181B2242
:106C7000BA1812781A708FE07B1D1B78032B49D14C
:106C80001F4B1B681B885B089BB2DAB21F23FB18E3
:106C90001B785BB20F21CB1A1D49CB5CDBB2D31A38
:106CA000DAB21C23FB181A701E23FB181C22BA1818
:106CB00012781A70124B1B685B885B089BB2DAB2C1
:106CC0001F23FB181B785BB21149CB5CDBB2D318D6
:106CD000DAB21D23FB181A70094B1B685B885B082E
:106CE0009BB2DAB21F23FB181B785BB20849CB5C5E
:106CF000DBB2D31ADAB21B23FB181A704CE0C04681
:106D0000300F0020ECBB0000F8BB000004BC00000A
:106D1000FCBD00007B1D1B78042B3DD1384B1B684C
:106D20001B885B089BB2DAB21F23FB181B785BB28F
:106D30003449CB5CDBB2D318DAB21E23FB181A70CD
:106D40002F4B1B681B885B089BB2DAB21F23FB1812
:106D50001B785BB22B49CB5CDBB2D31ADAB21C23B3
:106D6000FB181A70264B1B685B885B089BB2DAB273
:106D70001F23FB181B785BB20F21CB1A2149CB5C78
:106D8000DBB2D31ADAB21B23FB181A701D23FB18CF
:106D90001B22BA1812781A701E23FB1800229A566A
:106DA0001D23FB181B785BB2101C191CFFF7C2FDDA
:106DB0001F23FB181B785BB2002B0BDD1C23FB1879
:106DC00000229A561B23FB181B785BB2101C191C5F
:106DD000FFF7B0FD1F23FB181B78DBB20133DAB2DB
:106DE0001F23FB181A701F23FB181B785BB2072B9D
:106DF00000DCBBE6FBF73AF9BD4609B090BDC046E2
:106E0000300F0020FCBD000090B58BB002AF3A609F
:106E1000FB1D021C1A70BB1D0A1C1A701F23FB18D5
:106E200000221A701C23FB1800221A801A23FB1858
:106E300000221A80994B181CFBF78AFA974B1B68A3
:106E40001B885B089BB2203B1C1C944B1B685B8817
:106E50005B089BB2323B9149914A00930023019316
:106E6000081C111C0F22231CFBF7BCFC8B4B1B685E
:106E70001B885B089BB2283B1C1C884B1B685B88EB
:106E80005B089BB2233B8549864A0093002301930C
:106E9000081C111C0F22231CFBF7A4FCFB1D1B78F4
:106EA000002B17D07D4B1B681B885B089BB2283BCF
:106EB0001C1C7A4B1B685B885B089BB277497A4A3B
:106EC000009300230193081C111C0F22231CFBF7C5
:106ED00089FCDEE0BB1D1B78002B07D00823FA18C5
:106EE000724B101C191C03F0FFFE0DE0BB1D1B783C
:106EF00001225340DBB2002B06D00823FA186C4B5A
:106F0000101C191C03F0F0FE644B1B681B885B0807
:106F10009BB22D3B1C1C614B1B685B885B089BB2C2
:106F2000143B5E490822BA18009300230193081C01
:106F3000111C0F22231CFBF755FC584B1B681B88A8
:106F40005B089BB2373B1C1C544B1B685B885B087F
:106F50009BB2053B5149574A009300230193081CFB
:106F6000111C0F22231CFBF73DFC3B68181CFA2365
:106F7000990003F027FB031C181C03F063FE021C9E
:106F80001C23FB181A803B68181CFA23990003F095
:106F9000FFFB0B1C181C03F055FE031C181C64217E
:106FA00003F010FB031C1A1C1A23FB181A801C2365
:106FB000FB181A881A23FB181B88082178183E49E9
:106FC00003F092FE3B68002B03DA0823FB182D2206
:106FD0001A701C23FB181B88632B04D91F23FB1872
:106FE00010221A7008E01C23FB181B88092B03D9F8
:106FF0001F23FB1808221A70284B1B681B885B088C
:107000009BB2183B1A1C1F23FB181B78D41A234B66
:107010001B685B885B089BB20A3320490822BA18B8
:10702000009300230193081C111C0F22231CFBF763
:10703000D9FB1A4B1B681B885B089BB2373B1C1C97
:10704000164B1B685B885B089BB2283313491B4AAD
:10705000009300230193081C111C0F22231CFBF733
:10706000C1FB0E4B1B681B885B089BB2283B1C1C9A
:107070000A4B1B685B885B089BB232330749104A96
:10708000009300230193081C111C0F22231CFBF703
:10709000A9FBFAF7EBFFBD4609B090BD300F002009
:1070A00010BC00001CBC000028BC000034BC000068
:1070B00040BC00004CBC00005CBC000068BC000090
:1070C00078BC0000B0B588B002AF021C3960FB1D6F
:1070D0001A70564B181CFBF73BF9544B1B681B8866
:1070E0005B089BB2203B1C1C504B1B685B885B08F9
:1070F0009BB2323B4D494E4A009300230193081C3A
:10710000111C0F22231CFBF76DFB484B1B681B88CF
:107110005B089BB2283B1C1C444B1B685B885B08CC
:107120009BB2233B4149434A009300230193081C2F
:10713000111C0F22231CFBF755FB3C4B1B681B88C3
:107140005B089BB22C3B1C1C384B1B685B885B08A4
:107150009BB2143B3549384A009300230193081C25
:10716000111C0F22231CFBF73DFBFB1D1B78002B82
:1071700016D02E4B1B681B885B089BB2283B1C1C3F
:107180002A4B1B685B885B089BB228492B4A0093FB
:1071900000230193081C111C0F22231CFBF722FB68
:1071A000FB1D1B7801225340DBB2002B39D03B681A
:1071B000181CFA23990003F005FA031C1D1C3B68F8
:1071C000181CFA23990003F0E3FA0B1C181C03F0B7
:1071D00039FD031C181C642103F0F4F9031C1C1C6A
:1071E0000823FA18164B101C191C2A1C231C03F028
:1071F0007BFD0E4B1B681B885B089BB2323B1C1C43
:107200000A4B1B685B885B089BB208490822BA18C6
:10721000009300230193081C111C0F22231CFBF771
:10722000E1FAFAF723FFBD4606B0B0BD300F0020EB
:1072300010BC00001CBC000084BC000028BC000086
:1072400090BC000090B589B002AF041C081C111C52
:10725000FB1D221C1A70BB1D021C1A703B1D0A1C50
:107260001A801723FB1800221A70704B181CFBF7AA
:107270006FF86E4B1B681B885B089BB2203B1C1C85
:107280006A4B1B685B885B089BB2323B6749684A64
:10729000009300230193081C111C0F22231CFBF7F1
:1072A000A1FA624B1B681B885B089BB2343B1C1C19
:1072B0005E4B1B685B885B089BB25C495D4A009330
:1072C00000230193081C111C0F22231CFBF78AFAD0
:1072D000FB1D1B78002B30D0544B1B681B885B08B0
:1072E0009BB2343B1C1C514B1B685B885B089BB2F8
:1072F000233B4E49504A009300230193081C111C64
:107300000F22231CFBF76EFA484B1B681B885B0897
:107310009BB2343B1C1C454B1B685B885B089BB2D3
:10732000143B4249454A009300230193081C111C59
:107330000F22231CFBF756FA17E03C4B1B681B88F7
:107340005B089BB2283B1C1C384B1B685B885B08A6
:107350009BB2233B35493A4A009300230193081C12
:10736000111C0F22231CFBF73DFABB1D1B78002BC1
:107370000BD00823FA18334B101C191C03F0B4FC73
:107380001723FB1810221A700AE00823FA182E4B54
:10739000101C191C03F0A8FC1723FB180C221A70F0
:1073A000224B1B681B885B089BB21A1C1723FB1817
:1073B0001B78D41A1D4B1B685B885B089BB20F338C
:1073C0001A490822BA18009300230193081C111CC3
:1073D0000F22231CFBF706FA3B1D00229B5E002BAD
:1073E0001FD00823FA18194B101C191C03F07CFC41
:1073F0000E4B1B681B885B089BB2183B1C1C0B4B7D
:107400001B685B885B089BB2233308490822BA18C3
:10741000009300230193081C111C0F22231CFBF76F
:10742000E1F9FAF723FEBD4607B090BD300F00200A
:1074300010BC0000A4BC0000B4BC0000C4BC000030
:107440001CBC0000D4BC0000DCBC0000E4BB00009D
:10745000B0B588B002AF021C3960BB1D1A80754BF5
:10746000181CFAF775FF734B1B681B885B089BB2EF
:10747000203B1C1C6F4B1B685B885B089BB2323B3C
:107480006C496D4A009300230193081C111C0F22C4
:10749000231CFBF7A7F9674B1B681B885B089BB293
:1074A000343B1C1C634B1B685B885B089BB2233B13
:1074B0006049624A009300230193081C111C0F22AB
:1074C000231CFBF78FF95B4B1B681B885B089BB287
:1074D000383B1C1C574B1B685B885B089BB20F3BFF
:1074E0005449574A009300230193081C111C0F2292
:1074F000231CFBF777F93B68181CFA23990003F06B
:1075000061F8031C181C03F09DFB051C3B68181C4C
:10751000FA23990003F03CF90B1C181C03F092FBB2
:10752000031C181C642103F04DF8031C1C1C0823C9
:10753000FA18444B101C191C2A1C231C03F0D4FB02
:107540003B68002B03DA0823FB182D221A70394BF5
:107550001B681B885B089BB2203B1C1C354B1B68BF
:107560005B885B089BB233490822BA18009300235A
:107570000193081C111C0F22231CFBF733F908236D
:10758000FA18314B101C191C252203F0ADFB294BB6
:107590001B681B885B089BB2303B1C1C254B1B687F
:1075A0005B885B089BB2143322490822BA18009307
:1075B00000230193081C111C0F22231CFBF712F956
:1075C000BB1D1B88181C0A2102F06CFF031C9BB218
:1075D0001D1CBB1D1B88181C0A2102F0E9FF0B1C97
:1075E0009BB21C1C0823FA18184B101C191C2A1CCF
:1075F000231C03F079FB0F4B1B681B885B089BB2B5
:10760000143B1C1C0B4B1B685B885B089BB2233331
:1076100008490822BA18009300230193081C111C82
:107620000F22231CFBF7DEF8FAF720FDBD4606B05B
:10763000B0BDC046300F002010BC0000E0BC000010
:107640004CBC0000F0BC0000FCBC00000CBD000005
:10765000B0B588B002AF78603960714B181CFAF78A
:1076600077FE6F4B1B681B885B089BB2203B1C1C82
:107670006B4B1B685B885B089BB2323B6849694A6D
:10768000009300230193081C111C0F22231CFBF7FD
:10769000A9F8634B1B681B885B089BB2283B1C1C2A
:1076A0005F4B1B685B885B089BB2233B5C495E4A6F
:1076B000009300230193081C111C0F22231CFBF7CD
:1076C00091F8574B1B681B885B089BB2383B1C1C0E
:1076D000534B1B685B885B089BB20F3B5049534A76
:1076E000009300230193081C111C0F22231CFBF79D
:1076F00079F84B4B1B681B885B089BB2283B1C1C12
:10770000474B1B685B885B089BB214334449484A6B
:10771000009300230193081C111C0F22231CFBF76C
:1077200061F87B68181CFA23990002F04BFF031CD8
:10773000181C03F087FA051C7B68181C642102F0F2
:1077400041FF031C181C03F07DFA031C181C0A21BE
:1077500003F01EF80B1C1C1C0823FA18354B101CD8
:10776000191C2A1C231C03F0BFFA7B68002B03DAC8
:107770000823FB182D221A70294B1B681B885B08F5
:107780009BB2203B1C1C264B1B685B885B089BB292
:1077900023490822BA18009300230193081C111CE6
:1077A0000F22231CFBF71EF83B68181C0A2102F06D
:1077B00079FE031C181C03F045FA041C3B68181CD6
:1077C0000A2102F0F5FE0B1C181C03F03BFA011C09
:1077D0000823FA18184B0091101C191C2522231C91
:1077E00003F082FA0E4B1B681B885B089BB22C3B94
:1077F0001C1C0B4B1B685B885B089BB2233308493E
:107800000822BA18009300230193081C111C0F22B0
:10781000231CFAF7E7FFFAF729FCBD4606B0B0BD16
:10782000300F002010BC000018BD00004CBC000050
:1078300024BD0000F0BC000030BD0000B0B588B031
:1078400002AF78600A1CBB1C1A80674B181CFAF741
:107850007FFD654B1B681B885B089BB2203B1C1C93
:10786000614B1B685B885B089BB2323B5E495F4A99
:10787000009300230193081C111C0F22231CFAF70C
:10788000B1FF594B1B681B885B089BB22C3B1C1C2F
:10789000554B1B685B885B089BB2233B5249544A9B
:1078A000009300230193081C111C0F22231CFAF7DC
:1078B00099FF4D4B1B681B885B089BB2383B1C1C17
:1078C000494B1B685B885B089BB20F3B4649494AA2
:1078D000009300230193081C111C0F22231CFAF7AC
:1078E00081FF7B68181CFA23990002F06BFE031CD1
:1078F000181C03F0A7F9051C7B68181C642102F012
:1079000061FE031C181C03F09DF9031C181C0A21BE
:1079100002F03EFF0B1C1C1C0823FA18364B101CEF
:10792000191C2A1C231C03F0DFF97B68002B03DAE7
:107930000823FB182D221A702B4B1B681B885B0831
:107940009BB2203B1C1C284B1B685B885B089BB2CE
:1079500025490822BA18009300230193081C111C22
:107960000F22231CFAF73EFF1F4B1B681B885B0886
:107970009BB22C3B1C1C1C4B1B685B885B089BB29E
:10798000143319491D4A009300230193081C111C4C
:107990000F22231CFAF726FFBB1C1B880822B918EC
:1079A000174A081C111C1A1C03F09EF90E4B1B6889
:1079B0001B885B089BB2103B1C1C0B4B1B685B8835
:1079C0005B089BB2233308490822BA1800930023AE
:1079D0000193081C111C0F22231CFAF703FFFAF76E
:1079E00045FBBD4606B0B0BD300F002010BC000006
:1079F00040BD00004CBC0000F0BC00004CBD0000CD
:107A000058BD0000F0B58BB002AF78605A4B181C1F
:107A1000FAF79EFC0C23FA18584B101C191C03F0A3
:107A200063F9554B1B681B885B089BB2383B1C1CD9
:107A3000514B1B685B885B089BB2373B4E490C225D
:107A4000BA18009300230193081C111C1422231C54
:107A5000FAF7C8FE0C23FA18494B101C191C03F046
:107A600043F9454B1B681B885B089BB22C3B1C1CD5
:107A7000414B1B685B885B089BB22B3B3E490C2249
:107A8000BA18009300230193081C111C1422231C14
:107A9000FAF7A8FE0C23FA183A4B101C191C03F035
:107AA00023F9354B1B681B885B089BB2343B1C1CBD
:107AB000314B1B685B885B089BB2193B2E490C223B
:107AC000BA18009300230193081C111C1422231CD4
:107AD000FAF788FE7B68181C03F028F9061C264B71
:107AE0001B681B885B089BB21C1C234B24229B5CDD
:107AF000191C214B27229B5CCB181D1C7B68181C72
:107B000003F014F9031C6B435B08E31A1C1C1A4BAB
:107B10001B685B885B089BB217497A680093002357
:107B20000193081C111C321C231CFAF75BFE0C236A
:107B3000FA18154B101C191C03F0D6F80E4B1B68D5
:107B40001B885B089BB2343B1C1C0B4B1B685B887F
:107B50005B089BB22D3308490C22BA18009300230E
:107B60000193081C111C1422231CFAF73BFEFAF7A0
:107B70007DFABD4609B0F0BD300F0020C0BD000049
:107B8000D0BD0000DCBD0000ECBD000080B582B0BF
:107B900000AF786039607B681A683B68DA40131C74
:107BA00001221340181CBD4602B080BD80B582B0D2
:107BB00000AF78600649064A88235B00D3587A688C
:107BC000D2431A4088235B00CA50BD4602B080BD34
:107BD0000060004080B582B000AF78600649064A78
:107BE00088235B00D2587B681A4388235B00CA5005
:107BF000BD4602B080BDC0460060004080B582B086
:107C000000AF021C3960FB1D1A70FB1D1B78002B96
:107C10000DD0FB1D1B78012B09D0FB1D1B78022BFF
:107C200005D0FB1D1B78032B01D0FB1D1B78FB1D12
:107C30001A78131CDB009B189B001C33054A9A180A
:107C40003B68101C191CFFF7A1FF031C181CBD4644
:107C500002B080BD0060004080B500AF084B1B78CB
:107C6000002B03D1064B01221A7006E0044B1B784F
:107C7000012B02D1024B00221A70BD4680BDC046C6
:107C80005C0F002080B586B002AF214B1B78DBB2C1
:107C900001225340DBB2002B07D0FDF7BDFA1D4B8C
:107CA00000221A701A4B01221A701B4B1B78DBB290
:107CB000002B04D0FFF7D0FF174B00221A70154B92
:107CC0001A781649BB1D0093081C6021002301F09F
:107CD0003BFC031CFB600F4B1A78BB1D1B881BB2BF
:107CE000101C191C01F020FD031CBB60FB685A1E10
:107CF0009341D9B2074B1B785A1E9341DAB2BB6845
:107D0000081C111C1A1CFFF77FF8BD4604B080BD8B
:107D1000740F00205C0F0020710F002000A00040B5
:107D200090B587B002AF2E4B1B78DBB201225340D7
:107D3000DBB2002B0DD0FDF76FFA02F08BFB294967
:107D4000294A2A4B081C602101F052FF244B0122D2
:107D50001A70254B1A88254B1B88224912B21CB277
:107D60003B1C0093081C6021231C01F0E7FF031C4F
:107D7000BB60BB68002B26D13B687B600F23FB18E0
:107D800001221A7013E0174A3B1C101C60211A1CB8
:107D900001F0F0FD031CBB603B687A68D3187B6080
:107DA0000F23FB181A780F23FB1801321A700F23C8
:107DB000FB181B78042BE6D97B68181C052102F000
:107DC00001FC031C3B60BB685A1E9341DAB23B685E
:107DD000101C191CFFF776F9BD4605B090BDC046D2
:107DE000740F002000A000405E0F0020600F0020F4
:107DF00080B500AF034B181C6021012201F0CAFCC2
:107E0000BD4680BD00A0004080B500AF1020FFF748
:107E1000E1FEBD4680BDC04680B500AF1020FFF733
:107E2000C5FEBD4680BDC04680B500AFFFF7E0FF90
:107E3000FFF7EAFFBD4680BD80B500AF03200421F7
:107E4000FFF7DCFE031C5A1E9341DBB2181CBD4633
:107E500080BDC04680B584B000AF021CBB1D1A8037
:107E6000BB1D00229B5E181C02F0ECFE021CBA2314
:107E70009B019A4204DD0F23FB1801221A7003E0D4
:107E80000F23FB1800221A700F23FB181B78181CF5
:107E9000BD4604B080BDC04680B586B002AF7860F4
:107EA000104A7B680093101C60210022012301F01E
:107EB0004BFB031CBB60BB68002B04D00F23FB18DB
:107EC00001221A7003E00F23FB1800221A700F23FF
:107ED000FB181B785A1E9341DBB2181CBD4604B038
:107EE00080BDC04600A0004090B583B000AF204BDD
:107EF0001B78DBB201225340DBB2002B08D0FDF728
:107F00008BF902F0A7FAFFF78FFF194B01221A70C5
:107F1000BC1DFFF791FF031C2370BB1C181CFFF74F
:107F2000BBFF031C1A1C7B1D1A70BB1D1B78012292
:107F30005340DBB2002B08D0BB1C1B88FC1D1BB2BE
:107F4000181CFFF787FF031C23707B1D1B785A1E2C
:107F50009341D9B2BB1D1A78FB1D1B789BB21BB293
:107F6000081C111C1A1CFFF76DF9BD4603B090BD2B
:107F7000740F002080B500AF034B181C6021002255
:107F800001F008FCBD4680BD00A0004080B500AFF8
:107F9000FFF742FFFFF7EEFFBD4680BD80B582B020
:107FA00000AF021CFB1D1A70064BFA1D1278111C43
:107FB0001F220A40012191400A1C1A60BD4602B0EE
:107FC00080BDC04600E100E080B582B000AF021C79
:107FD000FB1D1A700649FB1D1B781A1C1F2313403A
:107FE00001229A40C0235B00CA50BD4602B080BD4A
:107FF00000E100E080B582B000AF78607B685B6A2A
:10800000181CBD4602B080BD80B582B000AF78605C
:1080100039607B683A681A62BD4602B080BDC046CE
:1080200080B582B000AF786039607B685A693B6880
:108030001A437B685A61BD4602B080BD80B582B0EC
:1080400000AF78607B689B69181CBD4602B080BD9C
:1080500080B582B000AF78600A1CFB1C1A70FB1C54
:108060001A787B685A60BD4602B080BD80B582B088
:1080700000AF094B181CFFF7E1FF031C7B60064AA9
:108080007B68101C191CFFF7BFFF044B01221A70FC
:10809000BD4602B080BDC04600200040620F0020F7
:1080A00080B586B000AF404B181C0121FBF7B2F839
:1080B0001023FB1800221A701023FB1800225A709C
:1080C0001023FB1800229A701023FB181F22DA706D
:1080D0001023FB1800221A711023FB1800225A717A
:1080E0000020FAF773FD031C1A1C1023FB18DA702A
:1080F0002E4B181C0021FAF731FD031C1A1C10230B
:10810000FB181A712A4A1023FB18101C191CFAF7C5
:1081100083FC3B1D00221A703B1D00225A703B1D40
:1081200000229A703B1D0022DA703B1D00221A715A
:108130003B1D00225A713B1D00229A713B1D0022FB
:10814000DA713B1D00221A723B1D00221A703B1D82
:1081500000225A703B1D0022DA703B1D04221A7166
:108160003B1D02229A703B1D00225A713B1D0022CA
:108170009A713B1D0022DA713B1D00221A720C4AD3
:108180003B1D101C191CFAF799FC094B181C012106
:10819000FFF746FF0420FFF717FF0420FFF7FEFE5E
:1081A000BD4606B080BDC04600A20400C0CF6A0034
:1081B0000020004080B500AFFDF72EF802F04AF92C
:1081C000FFF76EFFBD4680BD80B582B000AFFB1DDE
:1081D00000221A7000233B60FB1D00221A701AE077
:1081E000144B181C0121FFF733FFC046124B1B78BC
:1081F000DBB201225340DBB2002BF7D10D4B181C30
:10820000FFF7F8FE021C3B689B183B60FB1D1A78C9
:10821000FB1D01321A70FB1D1B78042BE0D93B6853
:10822000181C052102F03EF9031C9BB2181CBD4628
:1082300002B080BD00200040620F002080B584B0F5
:1082400000AF021CBB1D1A803B1D0A1C1A800E23A6
:10825000FB180D4A1A80BB1D1B880E22BA18128803
:1082600053435A003B1D1B88101C191C02F01AF9BD
:10827000031C1A1C0E23FB181B88D31ABB60BB6897
:10828000181CBD4604B080BDF64F000090B585B007
:1082900000AF0E23FB181F4A1A801F4B1B78DBB25E
:1082A00001225340DBB2002B04D0FFF783FF1A4BAF
:1082B00001221A700C23FC18FFF786FF031C238091
:1082C0000C23FB181B88FA2292005A430E23FB183A
:1082D0001B88101C191C02F075F9031C1A1C0A23B8
:1082E000FB181A800C23FB181A880E23FB181B8816
:1082F000101C191CFFF7A2FF031C7B600A23FB184C
:108300001A887B68101C191CFFF7A2F8BD4605B03F
:1083100090BDC046FF0F0000740F002080B582B0F2
:1083200000AF021CFB1D1A70064BFA1D1278111CBF
:108330001F220A40012191400A1C1A60BD4602B06A
:1083400080BDC04600E100E080B582B000AF021CF5
:10835000FB1D1A700649FB1D1B781A1C1F231340B6
:1083600001229A40131C80228B50BD4602B080BD72
:1083700000E100E080B582B000AF021CFB1D1A7066
:108380000649FB1D1B781A1C1F23134001229A402B
:10839000C0235B00CA50BD4602B080BD00E100E0D2
:1083A00080B582B000AF786039607B681A683B683E
:1083B000DA40131C01221340181CBD4602B080BDD8
:1083C00080B500AF044B044A126904218A431A6144
:1083D00030BFBD4680BDC04600ED00E080B582B034
:1083E00000AF021C3960FB1D1A70FB1D1B78002BAF
:1083F0000DD0FB1D1B78012B09D0FB1D1B78022B18
:1084000005D0FB1D1B78032B01D0FB1D1B78FB1D2A
:108410001A78131CDB009B189B001C33054A9A1822
:108420003B68101C191CFFF7BBFF031C181CBD4642
:1084300002B080BD0060004080B582B000AF7860BF
:108440000A1CFB1C1A707B680C4A934207D07B689D
:108450000B4A934203D07B680A4A934200D1C0463C
:10846000FB1C1B78002B03D07B6801225A6002E0C2
:108470007B6802225A60BD4602B080BD0000014008
:10848000000401400008014080B582B000AF786070
:1084900039607B683A689A61BD4602B080BDC046CB
:1084A00080B582B000AF786039607B68DB683A687D
:1084B000D2431A407B68DA60BD4602B080BDC04638
:1084C00080B582B000AF786039607B68DA683B685D
:1084D0001A437B68DA60BD4602B080BD80B582B0C9
:1084E00000AF78607B681B69181CBD4602B080BD78
:1084F00080B58AB000AF11200521FBF773F8032087
:10850000FBF790F92A4B181C0121FAF783FE294B3F
:10851000181C0121FAF77EFEC0239B030120191CC1
:1085200004220023FCF784FA1C23FA18224B111CA6
:108530001A1C0B23081C111C1A1C02F0C3FB10236D
:10854000FA181E4B111C1A1C0B23081C111C1A1C98
:1085500002F0B8FB1A4A1C23FB18101C00211A1C3D
:10856000FCF7D4FB164A1023FB18101C01211A1C1F
:10857000FCF7CCFB3B1C00221A6000225A60002250
:108580009A6000221A733B1C01225A703B1C032282
:10859000DA710220FFF7EEFE0220FFF7BFFE084A65
:1085A0003B1C101C191CFCF733FBBD460AB080BDF8
:1085B00000620400000204000CBE000018BE0000AF
:1085C0000000014080B500AFFCF726FE01F042FF3D
:1085D000FFF78EFFBD4680BD80B500AFFFF7F0FE10
:1085E000BD4680BD80B582B000AF0E4B181C112176
:1085F000FFF74AFF0B4B181C1121FFF761FFFB1D12
:1086000000221A7006E0FFF7E7FFFB1D1A78FB1D3A
:1086100001321A70FB1D1B78022BF4D9BD4602B043
:1086200080BDC0460000014080B500AF054B181C5E
:108630001121FFF735FF034B181C1121FFF724FF11
:10864000BD4680BD0000014080B584B000AF7860B9
:1086500039600023FB600A23FB18104A1A807A68ED
:108660003B689A4211D80A23FB181B887A68534347
:108670005B00181C396801F015FF031C1A1C0A2343
:10868000FB181B88D31AFB6003E00A23FB181B8826
:10869000FB60FB68181CBD4604B080BDF64F0000AF
:1086A00080B582B000AF786039607B68FA229200B2
:1086B0005343181C396801F0F5FE031C181CBD4615
:1086C00002B080BD80B500AF03200421FFF786FE15
:1086D000031C5A1E9341DBB2181CBD4680BDC04628
:1086E00090B587B000AF00233B610023FB60FB1C0B
:1086F00000221A70374B1B78DBB201225340DBB2E9
:10870000002B04D0FFF75EFF324B01221A70FFF7F7
:1087100069FF1723FB1800221A7017E0FFF75CFFB0
:108720002D4B1B683A69D3183B612C4B1B68FA68C8
:10873000D318FB602A4B1B78002B00D00BE01723CB
:10874000FB181A781723FB1801321A701723FB182D
:108750001B78042BE2D9FFF767FF214B1B78002B16
:1087600013D0FC1CFFF7AEFF031C2370FB1C1B780F
:10877000002B05D0FA239B00BB601A4B7B601FE0E7
:108780000023BB60184B7B601AE03A69FB68101C41
:10879000191CFFF785FF031CBB603B69181C0521F2
:1087A00001F080FE031C1C1CFB68181C052101F055
:1087B00079FE031C201C191CFFF746FF031C7B607D
:1087C0007A68BB68101C191CFEF742FFBD4607B053
:1087D00090BDC046740F0020640F0020680F002079
:1087E000630F0020F64F00000AB0FFFF80B582B093
:1087F00000AF144B181CFFF771FE021CBB1D1A8042
:10880000BB1D1B880122134003D00F4B01221A709D
:108810000FE0BB1D1B88102213400AD00A4B002218
:108820001A70084B5A6B094B1A60064B5A6C084B6E
:108830001A60044B181C1121FFF726FEBD4602B03A
:1088400080BDC04600000140630F0020680F00207B
:10885000640F002080B500AF0C4B181C0021FFF7FF
:10886000EBFD0B4B181C0021FAF7D4FC074B181C2E
:108870003121FFF715FE0220FFF766FD054B181C9E
:108880000021FAF7C7FCBD4680BDC046000001408C
:10889000000204000062040080B582B000AF021C38
:1088A000FB1D1A70064BFA1D1278111C1F220A407C
:1088B000012191400A1C1A60BD4602B080BDC0462D
:1088C00000E100E080B582B000AF021CFB1D1A7011
:1088D0000649FB1D1B781A1C1F23134001229A40D6
:1088E000131C80228B50BD4602B080BD00E100E029
:1088F00080B582B000AF021CFB1D1A700649FB1D3B
:108900001B781A1C1F23134001229A40C0235B00CE
:10891000CA50BD4602B080BD00E100E080B500AFA6
:10892000044B044A126904218A431A6130BFBD46D0
:1089300080BDC04600ED00E080B582B000AF786039
:1089400039607A683B6803331B01D3185B68181CD5
:10895000BD4602B080BDC04680B582B000AF786031
:108960000A1CFB1C1A707B680C4A934207D07B6878
:108970000B4A934203D07B680A4A934200D1C04617
:10898000FB1C1B78002B03D07B6801225A6002E09D
:108990007B6802225A60BD4602B080BD00000140E3
:1089A000000401400008014080B582B000AF78604B
:1089B00039607B683A689A61BD4602B080BDC046A6
:1089C00080B582B000AF786039607B68DB683A6858
:1089D000D2431A407B68DA60BD4602B080BDC04613
:1089E00080B582B000AF786039607B68DA683B6838
:1089F0001A437B68DA60BD4602B080BD80B582B0A4
:108A000000AF78607B681B69181CBD4602B080BD52
:108A100080B500AF0320042102220123FBF706FAF0
:108A2000BD4680BD80B500AF032004210122012393
:108A3000FBF7FCF9BD4680BD80B582B000AF194B95
:108A4000181CFFF7DBFF021CBB1D1A80BB1D1B8817
:108A50000122134002D0144B01221A70BB1D1B8847
:108A60001022134015D0104B00221A700D4B181C09
:108A70000021FFF761FF0B4B181C0021FFF75CFF83
:108A8000084B181C0021FFF757FF031C9AB2074B35
:108A90001A80044B181C1121FFF786FFBD4602B057
:108AA00080BDC046000401406E0F00206C0F002006
:108AB00080B588B000AF11200521FAF793FD03209F
:108AC000FAF7B0FE214B181C0121FAF7A3FB204B4B
:108AD000181C0121FAF79EFBC0239B030120191CDF
:108AE00004220023FBF7A4FF1423FA18194B111CCE
:108AF0001A1C0B23081C111C1A1C02F0E3F8164A5E
:108B00001423FB18101C00211A1CFCF7FFF83B1D56
:108B100000221A6000225A6000229A6000221A7312
:108B20003B1D01225A703B1D03229A710720FFF75B
:108B3000DFFE0720FFF7B0FE074A3B1D101C191C83
:108B4000FCF766F8BD4608B080BDC0460062040070
:108B50000012040024BE00000004014080B500AFF4
:108B6000FCF75AFB01F076FCFFF752FFFFF7A0FF7E
:108B7000BD4680BD80B500AF054B181C1121FFF725
:108B800013FF034B181C1121FFF72AFFBD4680BDC0
:108B90000004014080B500AF054B181C1121FFF700
:108BA0000FFF034B181C1121FFF7FEFEBD4680BDD1
:108BB0000004014080B584B000AF021CBB1D1A80C8
:108BC0000023FB6080231B01BB60BB1D1A88BB68B0
:108BD000D21A131C9B009B185B00FB60FB68181CDF
:108BE000BD4604B080BDC04680B500AFFFF796FE1D
:108BF000BD4680BD80B582B000AFFB1D00221A705B
:108C000016E0FFF7F1FF0F4B1B88FA1DF91D0978DD
:108C100011700D4A93420BD80A4B1B88FA1DF91D9F
:108C200009781170094A934202D9FB1D01221A707A
:108C3000FB1D1B7801225340DBB2002BE1D1BD4666
:108C400002B080BD6C0F002017100000880E0000DD
:108C5000B0B584B000AF051C0C1C101C191CBB1D4A
:108C60002A1C1A803B1D221C1A80BB1C021C1A8065
:108C70003B1C0A1C1A803B1D1C88BB1D1B88181C32
:108C8000702101F00FFC031C9BB2E218131CDB00E7
:108C90009B1ADB001A1CBB1D1B88101C191C01F041
:108CA00091FC031C0C3B1B029DB2BB1C1C88BB1D12
:108CB0001B88181C702101F0F5FB031C9BB2E21805
:108CC000131CDB009B1ADB001A1CBB1D1B88101C2D
:108CD000191C01F077FC031C0C3B1B019BB22A1CE6
:108CE00013439DB23B1C1C88BB1D1B88181C7021A4
:108CF00001F0D8FB031C9BB2E218131CDB009B1A8B
:108D0000DB001A1CBB1D1B88101C191C01F05AFC2F
:108D1000031C9BB20C3B9BB29BB22A1C13439AB21E
:108D20000E23FB181A800E23FB181B88181CBD4647
:108D300004B0B0BD90B589B000AF1C23FB18002271
:108D40001A803F4B1B78DBB201225340DBB2002B71
:108D500008D000200021FEF771FDFFF7FFFE384B21
:108D600001221A701F23FB1800221A7043E0FFF73C
:108D700001FFFFF73FFF334B1A883B1D1A801E236C
:108D8000FB1801221A7010E0FFF72EFF1E23FB18BC
:108D90001A782C4B19883B1D5200D1521E23FB1808
:108DA0001A781E23FB1801321A701E23FB181B7839
:108DB000072BE9D9FFF7EEFE3B1D18883B1D99886C
:108DC0003B1DDA883B1D1B891A243C19FFF740FF25
:108DD000031C23801C23FB181C22B9181A22BA1862
:108DE000098812888A181A801F23FB181A781F23F3
:108DF000FB1801321A701F23FB181B78042BB6D9FD
:108E00001C23FB181B88181C052101F04BFB031CBD
:108E10009BB2181CFFF7CEFE031C7B611C23FB18C2
:108E20001B88181C052101F03DFB031C9BB27A69CD
:108E3000101C191CFEF702FDBD4609B090BDC046CE
:108E4000740F00206C0F002080B500AFFFF7EAFD23
:108E50000C4B181C0021FFF77FFD0A4B181C312119
:108E6000FFF7AEFD0720FFF72DFD074B181C002173
:108E7000FAF7D0F9054B181C0021FAF7CBF9BD46DB
:108E800080BDC046000401400012040000620400DE
:108E900090B58DB000AFF860081C111C7B600B23EF
:108EA000FB18021C1A700A23FB180A1C1A700B23E9
:108EB000FB181B789AB21823FB181A801823FB188A
:108EC00004225A801423FB180A22BA1812781A7046
:108ED0001823FB181422BA185A601823FB18012211
:108EE0001A811823FB187A68DA601823FB1801220C
:108EF0001A822F23FC18FA681823FB18101C191C5F
:108F0000F7F7E2FE031C23702F23FB181B785BB2DC
:108F1000002B07D07B68FF221A702F23FB181B78C9
:108F20005BB200E00023181CBD460DB090BDC046EA
:108F300090B58BB000AF78600C1C101C191CFB1C8A
:108F4000221C1A70BB1C021C1A707B1C0A1C1A7093
:108F5000FB1C1B789AB21023FB181A801023FB18F5
:108F600001225A800C23FB18BA1C12781A700C23A9
:108F7000FB187A1C12785A701023FB180C22BA18AE
:108F80005A601023FB1802221A811023FB180822B2
:108F9000BA18DA601023FB1800221A822723FC1863
:108FA0007A681023FB18101C191CF7F78DFE031CA0
:108FB00023702723FB181B785BB2002B04D02723D8
:108FC000FB181B785BB200E00023181CBD460BB0F9
:108FD00090BDC04680B586B000AFF8607A600B23C4
:108FE000FB180A1C1A701223FB1800221A700023A7
:108FF0007B611323FB1800221A70F9680B23FB18FE
:109000001A781223FB18081C111CC122FFF740FF1D
:10901000031C7B611223FB181A781323FB18D20957
:109020001A701223FB181B781A1C7F2313401B0293
:109030009AB27B681A80F9680B23FB181A781223FE
:10904000FB18081C111CC222FFF722FF021C7B69BF
:1090500013437B617B681A881223FB181B789BB231
:1090600013439AB27B681A807B681B889BB2094ABB
:10907000944663449BB29AB27B681A801323FB1810
:109080001B78002B01D1FD237B617B69181CBD4639
:1090900006B080BD00C0FFFF90B585B000AF78601E
:1090A0000A1CFB1C1A700023FB607968FB1C1A78F1
:1090B0000B23FB18081C111CC922FFF7E9FE031C37
:1090C000FB600B23FB181B7801229343DAB20B23BE
:1090D000FB181A700B23FB181C787A68FB1C1B7892
:1090E000101C191CC922231CFFF722FF021CFB685D
:1090F0001343FB607968FB1C1A780B23FB18081CD0
:10910000111CC422FFF7C4FE021CFB681343FB6062
:109110000B23FB181B7801221343DAB20B23FB1835
:109120001A700B23FB181C787A68FB1C1B78101C28
:10913000191CC422231CFFF7FBFE021CFB6813430F
:10914000FB60FB68181CBD4605B090BD90B585B0AE
:1091500000AF78600A1CFB1C1A700023FB60796862
:10916000FB1C1A780B23FB18081C111CC922FFF7E3
:109170008FFE031CFB600B23FB181B78DBB21A1C51
:1091800003239A43131CDBB21A1C01231343DBB2E3
:10919000DAB20B23FB181A700B23FB181C787A68C1
:1091A000FB1C1B78101C191CC922231CFFF7C0FED6
:1091B000021CFB681343FB607968FB1C1A780B23C5
:1091C000FB18081C111CC422FFF762FE031CFB6085
:1091D0000B23FB181B7807229343DAB20B23FB18EF
:1091E0001A700B23FB181C787A68FB1C1B78101C68
:1091F000191CC422231CFFF79BFE021CFB681343AF
:10920000FB60FB68181CBD4605B090BD90B58BB0E7
:1092100000AF78600A1CFB1C1A70FB1C1B789AB20A
:109220001023FB181A801023FB1801225A801023E8
:10923000FB180C22BA185A601023FB1800221A815E
:109240001023FB180822BA18DA601023FB1800223A
:109250001A822723FC187A681023FB18101C191C8B
:10926000F7F732FD031C23702723FB181B785BB232
:10927000002B04D02723FB181B785BB200E00023EF
:10928000181CBD460BB090BD80B586B000AFF8602D
:10929000081C111C7B600B23FB18021C1A700A238C
:1092A000FB180A1C1A70F9680B23FB181A78132391
:1092B000FB18081C111CE322FFF7EAFD031C7B616D
:1092C0001323FB181B781A1C0123134001D0FE2323
:1092D00032E0F9680B23FB181A780A23FB181B7875
:1092E000081C111CE122FFF723FE021C7B691343BB
:1092F0007B61FA680B23FB181B78101C191CE322F6
:109300000223FFF715FE021C7B6913437B61F9689A
:109310000B23FB181A781323FB18081C111CE222DC
:10932000FFF7B6FD021C7B6913437B611323FB1817
:109330001A787B681A707B69181CBD4606B080BD20
:1093400090B587B000AF7860081C111CFB1C021C94
:109350001A70BB1C0A1C1A70BB1C1B78002B04D192
:109360001723FB1821221A7007E0BB1C1B78012B66
:1093700003D11723FB1827221A701723FB181B7819
:109380001722BA18591C11707968FA1C12780F202C
:109390003C18081C111C1A1C231CFFF775FF031C2A
:1093A0003B610F23FB181C787A68FB1C1B78101C90
:1093B000191CCA22231CFFF7BBFD021C3B69134387
:1093C0003B611723FB181B781722BA18591C117020
:1093D0007968FA1C12780F203C18081C111C1A1C02
:1093E000231CFFF751FF021C3B6913433B610F2312
:1093F000FB181C787A68FB1C1B78101C191CCB22EC
:10940000231CFFF795FD021C3B6913433B611723A7
:10941000FB181B781722BA18591C11707968FA1CAE
:1094200012780F203C18081C111C1A1C231CFFF773
:109430002BFF021C3B6913433B610F23FB181C7875
:109440007A68FB1C1B78101C191CCC22231CFFF70C
:109450006FFD021C3B6913433B611723FB181B780C
:109460001722BA18591C11707968FA1C12780F204B
:109470003C18081C111C1A1C231CFFF705FF021CBA
:109480003B6913433B610F23FB181C787A68FB1C74
:109490001B78101C191CCE22231CFFF749FD021C4F
:1094A0003B6913433B611723FB181B781722BA183B
:1094B000591C11707968FA1C12780F203C18081C8E
:1094C000111C1A1C231CFFF7DFFE021C3B6913430F
:1094D0003B610F23FB181C787A68FB1C1B78101C5F
:1094E000191CCF22231CFFF723FD021C3B691343E9
:1094F0003B611723FB181B781722BA18591C1170EF
:109500007968FA1C12780F203C18081C111C1A1CD0
:10951000231CFFF7B9FE021C3B6913433B610F2379
:10952000FB181C787A68FB1C1B78101C191CD022B5
:10953000231CFFF7FDFC021C3B6913433B613B69A5
:10954000181CBD4607B090BD90B585B000AF7860DF
:109550000C1C101C191CFB1C221C1A70BB1C021CAE
:109560001A707B1C0A1C1A700B23FB1800221A703D
:109570000023FB607A68FB1C1B78101C191CFFF78A
:1095800045FE031CFB607968FB1C1A780B23FB1853
:10959000081C111CC422FFF77BFC021CFB68134350
:1095A000FB600B23FB181B78DBB21A1C0F239A43BA
:1095B000131CDBB21A1C02231343DBB2DAB20B23F7
:1095C000FB181A700B23FB181C787A68FB1C1B789D
:1095D000101C191CC422231CFFF7AAFC021CFB68E8
:1095E0001343FB607968FB1C1A78BB1C1B78081CB2
:1095F000111C1A1CFFF7A4FE021CFB681343FB603E
:109600007A68FB1C1B78101C191CCD220E23FFF757
:109610008FFC021CFB681343FB607968FB1C1A7803
:109620000B23FB18081C111CC422FFF731FC021C81
:10963000FB681343FB600B23FB181B78DBB21A1C7F
:109640000F239A43131CDBB21A1C04231343DBB20F
:10965000DAB20B23FB181A700B23FB181C787A68FC
:10966000FB1C1B78101C191CC422231CFFF760FC78
:10967000021CFB681343FB607968FB1C1A780B2300
:10968000FB18081C111CC422FFF702FC021CFB681B
:109690001343FB600DE07968FB1C1A780B23FB1861
:1096A000081C111CC422FFF7F3FB021CFB681343C8
:1096B000FB600B23FB181B78DBB25BB2002B02DADA
:1096C000FB68002BE7D07968FB1C1A783B6A081C02
:1096D000111C1A1CFFF77EFC021CFB681343FB6085
:1096E0007B1C1B78002B0BD17A68FB1C1B78101C91
:1096F000191CFFF7D1FC021CFB681343FB600EE052
:109700007B1C1B78012B0AD17A68FB1C1B78101C70
:10971000191CFFF71BFD021CFB681343FB60FB6871
:10972000181CBD4605B090BD80B584B000AF021CCA
:10973000FB1D1A703B1D0A1C1A800023FB60FB1DD9
:109740001B78002B0ED13B1D00229A5E131C5B017F
:109750009B1A9B009B18181C642100F033FF031C0C
:10976000FB6011E0FB1D1B78012B0DD13B1D00227E
:109770009A5E131C5B019B1A9B009B18181C0A2104
:1097800000F020FF031CFB60FB68181CBD4604B002
:1097900080BDC04680B584B000AF7860081C111C45
:1097A000FB1C021C1A70BB1C0A1C1A700023FB60F5
:1097B0007A68FB1C1B78101C191CFFF727FD031C83
:1097C000FB60BB1C1B78002B0BD17A68FB1C1B7841
:1097D000101C191CFFF760FC021CFB681343FB60A4
:1097E0000EE0BB1C1B78012B0AD17A68FB1C1B788E
:1097F000101C191CFFF7AAFC021CFB681343FB603A
:10980000FB68181CBD4604B080BDC04690B585B04D
:1098100000AF78600A1CFB1C1A700023FB607A689A
:10982000FB1C1B78101C191CFFF7F0FC031CFB60D1
:109830007968FB1C1A780B23FB18081C111CC42226
:10984000FFF726FB021CFB681343FB600B23FB188E
:109850001B780A221343DAB20B23FB181A700B236E
:10986000FB181C787A68FB1C1B78101C191CC4227E
:10987000231CFFF75DFB021CFB681343FB600B23FB
:10988000FB18FF221A700B23FB181C787A68FB1C4C
:109890001B78101C191CC622231CFFF749FB021C55
:1098A000FB681343FB600B23FB1892221A700B23F7
:1098B000FB181C787A68FB1C1B78101C191CC7222B
:1098C000231CFFF735FB021CFB681343FB60796820
:1098D000FB1C1A780B23FB18081C111CC922FFF76C
:1098E000D7FA021CFB681343FB600B23FB181B78A1
:1098F00001221343DAB20B23FB181A700B23FB1857
:109900001C787A68FB1C1B78101C191CC922231CAC
:10991000FFF70EFB021CFB681343FB607968FB1C1E
:109920001A780B23FB18081C111CC422FFF7B0FA8D
:10993000021CFB681343FB600B23FB181B780222FD
:109940009343DAB20B23FB181A700B23FB181C7815
:109950007A68FB1C1B78101C191CC422231CFFF7FF
:10996000E7FA021CFB681343FB60FB68181CBD464A
:1099700005B090BD90B58BB000AFF8607A600B2356
:10998000FB180A1C1A7000237B622223FB1800229A
:109990001A80FA680B23FB181B78101C191CFFF7A0
:1099A00035FC031C7B62F9680B23FB181A7817231C
:1099B000FB18081C111CC422FFF76AFA021C7B6A00
:1099C00013437B621723FB181B78DBB21A1C0F238F
:1099D0009A43131CDBB21A1C02231343DBB2DAB224
:1099E0001723FB181A701723FB181C78FA680B232F
:1099F000FB181B78101C191CC422231CFFF798FAB3
:109A0000021C7B6A13437B622223FB181B88DCB297
:109A1000FA680B23FB181B78101C191CCD22231C81
:109A2000FFF786FA021C7B6A13437B62F9680B23FB
:109A3000FB181A781723FB18081C111CC322FFF708
:109A400027FA021C7B6A13437B621723FB181B78DF
:109A5000DBB21A1C07239A43131CDBB21A1C012326
:109A60001343DBB2DAB21723FB181A701723FB1863
:109A70001C78FA680B23FB181B78101C191CC322D6
:109A8000231CFFF755FA021C7B6A13437B62F968BB
:109A90000B23FB181A781723FB18081C111CC4226F
:109AA000FFF7F6F9021C7B6A13437B621723FB184E
:109AB0001B78DBB21A1C07239A43131CDBB21A1C57
:109AC00004231343DBB2DAB21723FB181A701723EF
:109AD000FB181C78FA680B23FB181B78101C191C48
:109AE000C422231CFFF724FA021C7B6A13437B6207
:109AF000F9680B23FB181A781623FB18081C111C95
:109B0000C122FFF7C5F9021C7B6A13437B62F96827
:109B10000B23FB181A781523FB18081C111CC222F2
:109B2000FFF7B6F9021C7B6A13437B62FA680B23CA
:109B3000FB181B78101C191CFFF7AEFA021C7B6A7D
:109B400013437B621623FB181A782123FB18D209D2
:109B50001A702123FB181B78002B01D1FD233AE05A
:109B60001623FB181B781A1C7F2313401A021E238E
:109B7000FB181A801E23FB1800229B5E1522BA18C0
:109B800012781343DA101E23FB181A801E23FB18C9
:109B900000229B5E1E22BA180021525E5343104AD7
:109BA0005343181C0F4900F00DFD031C1C1C1E2301
:109BB000FB1800229B5E0C4A5343181C642100F0E2
:109BC00001FD031CE318094A94466344BB617B68AA
:109BD000BA691A607B6A181CBD460BB090BDC046BE
:109BE00081FEFFFFA0860100DE3E000008BBFBFFF8
:109BF00090B587B000AFF8607A603B600B23FB182C
:109C00000A1C1A7000237B611323FB181D221A7093
:109C10001223FB181E221A70FA680B23FB181B78FC
:109C2000101C191CFFF7F2FA031C7B61F9680B2367
:109C3000FB181A781123FB18081C111CC422FFF70B
:109C400027F9021C7B6913437B611123FB181B78E6
:109C5000DBB21A1C0F239A43131CDBB21A1C02231B
:109C60001343DBB2DAB21123FB181A701123FB186D
:109C70001C78FA680B23FB181B78101C191CC422D3
:109C8000231CFFF755F9021C7B6913437B61F868BD
:109C90000B23FB1819781323FB181A781123FB18D0
:109CA000FFF7F2FA021C7B6913437B611123FB1857
:109CB0001B78DBB25BB2FA2292005343002B00DA2E
:109CC0000F331B119AB27B681A80F8680B23FB18BC
:109CD00019781223FB181A781123FB18FFF7D4FA0E
:109CE000021C7B6913437B611123FB181B78DBB2D9
:109CF0005BB2FA2292005343002B02DA0E4A9446DA
:109D00006344DB129BB2FA229200944663449BB2F6
:109D10009AB23B681A80FA680B23FB181B78101C58
:109D2000191CFFF7B9F9021C7B6913437B617B693E
:109D3000181CBD4607B090BDFF07000090B58BB062
:109D400000AFF8600C1C101C191C0B23FB18221C04
:109D50001A700823FB18021C1A80BB1D0A1C1A80EB
:109D600000237B622223FB1800221A80FA680B234F
:109D7000FB181B78101C191CFFF748FA031C7B62A8
:109D8000F9680B23FB181A781323FB18081C111C05
:109D9000C422FFF77DF8021C7B6A13437B62132306
:109DA000FB181B78DBB21A1C0F239A43131CDBB27F
:109DB0001A1C02231343DBB2DAB21323FB181A7006
:109DC0001323FB181C78FA680B23FB181B78101C54
:109DD000191CC422231CFFF7ABF8021C7B6A134337
:109DE0007B622223FB181B88DCB2FA680B23FB186A
:109DF0001B78101C191CCD22231CFFF799F8021C9C
:109E00007B6A13437B62F9680B23FB181A781323D0
:109E1000FB18081C111CC322FFF73AF8021C7B6ACE
:109E200013437B621323FB181B78DBB21A1C072336
:109E30009A43131CDBB21A1C01231343DBB2DAB2C0
:109E40001323FB181A701323FB181C78FA680B23D2
:109E5000FB181B78101C191CC322231CFFF768F881
:109E6000021C7B6A13437B62F9680B23FB181A7888
:109E70001323FB18081C111CC422FFF709F8021C4D
:109E80007B6A13437B621323FB181B78DBB21A1C1B
:109E900007239A43131CDBB21A1C04231343DBB2BF
:109EA000DAB21323FB181A701323FB181C78FA6814
:109EB0000B23FB181B78101C191CC422231CFFF752
:109EC00037F8021C7B6A13437B62F9680B23FB188B
:109ED0001A781223FB18081C111CC122FEF7D8FFA8
:109EE000021C7B6A13437B62F9680B23FB181A7808
:109EF0001123FB18081C111CC222FEF7C9FF021C0B
:109F00007B6A13437B62FA680B23FB181B78101CD7
:109F1000191CFFF7C1F8021C7B6A13437B621223F2
:109F2000FB181A782123FB18D2091A702123FB1879
:109F30001B78002B01D1FD234BE01223FB181B786B
:109F40001A1C7F2313401A021E23FB181A801E239B
:109F5000FB1800229B5E1122BA1812781343DA1004
:109F60001E23FB181A801E23FB1800229B5E1E2254
:109F7000BA180021525E5343184A5343181C18491B
:109F800000F020FB031C1C1C1E23FB1800229B5E00
:109F9000144A5343181C642100F014FB031CE318FB
:109FA000114A94466344BB61BB1D00229B5EBA69A3
:109FB0005A430823FB1800215B5ED318181CFA23B0
:109FC000990000F0FFFA031C7B61BB6B7A691A6091
:109FD0007B6A181CBD460BB090BDC04681FEFFFFDA
:109FE000A0860100DE3E000008BBFBFF80B582B00A
:109FF00000AF021CFB1D1A70064BFA1D1278111CD3
:10A000001F220A40012191400A1C1A60BD4602B07D
:10A0100080BDC04600E100E080B582B000AF021C08
:10A02000FB1D1A700649FB1D1B781A1C1F231340C9
:10A0300001229A40C0235B00CA50BD4602B080BDD9
:10A0400000E100E080B582B000AF786039607B68E5
:10A050001A683B68DA40131C01221340181CBD46E5
:10A0600002B080BD80B582B000AF78603960094829
:10A07000084A92235B00D3583A68D2431A407B685F
:10A0800039680B401A4392235B00C250BD4602B0B0
:10A0900080BDC0460060004080B582B000AF7860EF
:10A0A00003498E235B007A68CA50BD4602B080BD6A
:10A0B0000060004080B500AF034A8A235B00D3589C
:10A0C000181CBD4680BDC0460060004080B582B00F
:10A0D00000AF021C3960FB1D1A70FB1D1B78002BA2
:10A0E0000DD0FB1D1B78012B09D0FB1D1B78022B0B
:10A0F00005D0FB1D1B78032B01D0FB1D1B78FB1D1E
:10A100001A78131CDB009B189B001C33054A9A1815
:10A110003B68101C191CFFF795FF031C181CBD465B
:10A1200002B080BD0060004090B585B002AF041C55
:10A130003960101C191CFB1D221C1A70BB1D021C4F
:10A140001A707B1D0A1C1A70FB1D187839683A6852
:10A15000BB1D1C787B1D1B7800931823FB181B78F4
:10A160000193231CF9F7DEFDBD4603B090BDC04648
:10A1700080B582B000AF094B1B687B607B681B0E0B
:10A18000812B08D8064B074A1A60074B064A12680B
:10A1900006490A401A60BD4602B080BDFC81E00F4E
:10A1A00018600C4005000004E4800C40FFFFFFFE37
:10A1B00080B500AFFFF7DCFF11200521F9F712FA97
:10A1C0000320F9F72FFB00F07DF800F069F8FBF7AA
:10A1D000B1FF00F043F81A4B1B78DBB2082B1FD8F5
:10A1E0009A00184BD3181B689F46FBF703FE1BE031
:10A1F000FBF72EF818E0FBF7B7FC15E0FDF742FD82
:10A2000012E0FDF78DFD0FE0FDF76EFE0CE0FEF7AE
:10A210003DF809E0FEF764FA06E0FEF78BFD03E087
:10A22000074B00221A70C046074B1B78DBB2012295
:10A230005340DBB2002B02D00120F9F7B1FCCAE792
:10A240006F0F002030BE0000710F002080B582B07B
:10A2500000AF78603960BD4602B080BD90B583B074
:10A2600002AF002001210022F9F73EFBF6F716FEAF
:10A27000094B181CF6F7CAFD074B1968FA239A0018
:10A28000064C00230093081C0121231CF6F75CFEFA
:10A29000BD4601B090BDC046980F00204DA2000001
:10A2A00090B587B000AF3B1C054A13CA13C313CA4D
:10A2B00013C33B1C181CF6F793FCBD4607B090BDBA
:10A2C00054BE000080B582B002AF2E4B181C012195
:10A2D000F8F7A0FF03200321FFF7C4FE02200921A5
:10A2E00002220123F9F7A2FD012300930220092194
:10A2F00000220123FFF718FF02200A210222012376
:10A30000F9F794FD0123009302200A210022012382
:10A31000FFF70AFF0220002101220123F9F786FD41
:10A320000220012101220123F9F780FD002300937F
:10A330000220002101220123FFF7F6FE00230093F3
:10A340000220012101220123FFF7EEFE0320042158
:10A3500001220023F9F76AFD002300930320042162
:10A3600001220123FFF7E0FE0120FFF755FE012047
:10A37000FFF73CFE0620FFF74FFE0620FFF736FEF4
:10A38000BD4680BD0082040080B582B000AFFFF7FB
:10A3900091FE031C7B607B68181CFFF77DFE7A68CA
:10A3A00080239B0013401AD0184B1B78DBB2002B84
:10A3B00003D1174B01221A7011E0144B1B78DBB24A
:10A3C000012B07D100F054F8031E03D0114B0122DA
:10A3D0001A7004E00D4B00221A7000F057F87A68EA
:10A3E0008023DB00134002D00B4B01221A707B68E4
:10A3F0000322134007D0054B1B78DBB2002B02D1A0
:10A40000064B01221A70BD4602B080BD6F0F0020BE
:10A41000700F0020720F0020710F0020730F0020BA
:10A4200080B500AFFFF7B0FFBD4680BD80B500AF7F
:10A43000FFF7AAFFBD4680BD80B582B002AF012301
:10A44000009302200A2100220123FFF76DFEBD4682
:10A4500080BDC04680B582B002AF002300930220C9
:10A460000A2100220123FFF75FFEBD4680BDC046E2
:10A4700080B500AF02200A21FFF728FE031C5A42D4
:10A480005341DBB2181CBD4680BDC04680B500AF4D
:10A49000FBF7E8FAFDF77AFDFEF7DCF9FEF7D4FCEE
:10A4A000BD4680BD002243088B4274D303098B4212
:10A4B0005FD3030A8B4244D3030B8B4228D3030C94
:10A4C0008B420DD3FF22090212BA030C8B4202D336
:10A4D0001212090265D0030B8B4219D300E0090A5E
:10A4E000C30B8B4201D3CB03C01A5241830B8B4267
:10A4F00001D38B03C01A5241430B8B4201D34B0350
:10A50000C01A5241030B8B4201D30B03C01A5241B4
:10A51000C30A8B4201D3CB02C01A5241830A8B4239
:10A5200001D38B02C01A5241430A8B4201D34B0222
:10A53000C01A5241030A8B4201D30B02C01A524186
:10A54000CDD2C3098B4201D3CB01C01A524183093A
:10A550008B4201D38B01C01A524143098B4201D374
:10A560004B01C01A524103098B4201D30B01C01A9F
:10A570005241C3088B4201D3CB00C01A5241830819
:10A580008B4201D38B00C01A524143088B4201D346
:10A590004B00C01A5241411A00D2014652411046A6
:10A5A0007047FFE701B5002000F0FCF802BDC0468F
:10A5B0000029F7D003B5FFF775FF0EBC4243891A97
:10A5C0001847C04603460B437FD4002243088B4202
:10A5D00074D303098B425FD3030A8B4244D3030B2A
:10A5E0008B4228D3030C8B420DD3FF22090212BAEF
:10A5F000030C8B4202D31212090265D0030B8B426B
:10A6000019D300E0090AC30B8B4201D3CB03C01A54
:10A610005241830B8B4201D38B03C01A5241430B2F
:10A620008B4201D34B03C01A5241030B8B4201D31F
:10A630000B03C01A5241C30A8B4201D3CB02C01A8A
:10A640005241830A8B4201D38B02C01A5241430A02
:10A650008B4201D34B02C01A5241030A8B4201D3F1
:10A660000B02C01A5241CDD2C3098B4201D3CB0198
:10A67000C01A524183098B4201D38B01C01A524147
:10A6800043098B4201D34B01C01A524103098B424B
:10A6900001D30B01C01A5241C3088B4201D3CB0036
:10A6A000C01A524183088B4201D38B00C01A524119
:10A6B00043088B4201D34B00C01A5241411A00D2C9
:10A6C00001465241104670475DE0CA0F00D0494232
:10A6D000031000D34042534000229C4603098B42A2
:10A6E0002DD3030A8B4212D3FC22890112BA030A2A
:10A6F0008B420CD3890192118B4208D389019211AC
:10A700008B4204D389013AD0921100E08909C30930
:10A710008B4201D3CB01C01A524183098B4201D332
:10A720008B01C01A524143098B4201D34B01C01A1D
:10A73000524103098B4201D30B01C01A5241C30895
:10A740008B4201D3CB00C01A524183088B4201D304
:10A750008B00C01A5241D9D243088B4201D34B001F
:10A76000C01A5241411A00D20146634652415B1061
:10A77000104601D34042002B00D549427047634642
:10A780005B1000D3404201B5002000F00BF802BD81
:10A790000029F8D003B5FFF715FF0EBC4243891A14
:10A7A0001847C0467047C0461C2101231B0498422D
:10A7B00001D3000C10391B0A984201D3000A083952
:10A7C0001B09984201D30009043902A2105C401809
:10A7D0007047C046040302020101010100000000AD
:10A7E00000000000002B11D1002A0FD1002900D158
:10A7F000002802D00021C943081C07B4024802A166
:10A800004018029003BDC0469DFFFFFF03B4684699
:10A8100001B5029800F04CF8019B9E4602B00CBCBA
:10A820007047C046F0B54F46464605042D0C2C1C1B
:10A83000C0B41704160C3F0C9946030C7C437543B7
:10A840005F4373437D19260CAD199C46AF4203D973
:10A8500080235B029846C4444B465143434324043F
:10A860002E0C240C2D0466442C1959188919201C0F
:10A870000CBC90469946F0BDF0B583B0161C1F1C69
:10A880000090019100F02EF8041C0D1C221C2B1CC2
:10A89000301C391CFFF7C6FF009A019B121A8B412E
:10A8A0000899201C0A604B60291C03B0F0BDC0460B
:10A8B000F0B5141C83B01D1C0090019100F00AF942
:10A8C000221C2B1C061C0F1CFFF7ACFF009A019BDF
:10A8D000121A8B410899301C0A604B60391C03B076
:10A8E000F0BDC046F0B544465F4656464D46F0B40E
:10A8F0001C1C85B0002900DAA9E00F1C0021061CF1
:10A900008846101C191C002C00DA97E0341C3D1CF2
:10A9100082468946B94273D870D04946504600F005
:10A9200085F98346391C301C00F080F95B46181A03
:10A93000031C8346203B9C4600D59CE0002300225C
:10A9400051460092019363469940019151468140DE
:10A95000019B0091BB4200D983E000D17EE0009AC8
:10A96000019B341C3D1CA41A9D416346002B00DA58
:10A970009AE0002600270296039701369E40039630
:10A98000012686400296002800D171E00099019AC4
:10A99000D30799464B464E081E4357080023012211
:10A9A0000CE0AF4201D1A6420AD8A41BBD41241934
:10A9B0006D410138A4185D41002806D0AF42F0D99E
:10A9C000013824196D410028F8D12022029E039FEE
:10A9D0005B46524236196F4199185AD4281CC84018
:10A9E0002C1C5B46DC40002968DB041C8C40231CCB
:10A9F00059468840021CB61A9F4103E0B0428CD9E8
:10AA00000026002741464B1E9941002300910193E7
:10AA1000009A019B002554429D41331C6340181C41
:10AA20003B1C6B40191C009B019CC018614105B088
:10AA30003CBC90469946A246AB46F0BD4346DB433C
:10AA40000C1C9846131C00215842A1415EE70027C8
:10AA500046428F4101214942884652E7B14200D81F
:10AA60007DE70026002702960397002800D08DE797
:10AA7000029E039FC6E720215346091ACB400022BD
:10AA8000191C0023009201934B4683400B43019312
:10AA90005CE75A4620239B1A2A1C9A40201C131C50
:10AAA0005A46D04018439BE720260027331A002639
:10AAB000029603970127DF40039761E75B46202159
:10AAC0005D46C91A031CAC40CB40191C231C0B4328
:10AAD0008EE7C046F0B545464E465746E0B4041CE6
:10AAE00082B00D1C914698468B4262D85FD0414699
:10AAF000484600F09BF8291C061C201C00F096F824
:10AB00002023311A5B428A46C81865D44B468340DD
:10AB10001F1C4B468B401E1CAF4258D855D0A41B5F
:10AB2000BD41002800DA77E0002200230092019363
:10AB300001328240019201238B40009300293CD0D6
:10AB4000FB079846404672087B080243012600270F
:10AB50000CE0AB4201D1A2420AD8A41A9D412419AB
:10AB60006D410139A4197D41002906D0AB42F0D9CD
:10AB7000013924196D410029F8D12022009801994A
:10AB800053465242001969419E183AD42F1CF7408F
:10AB90005346DD40002E29DB3C1CB440231C5446A8
:10ABA000A7403A1C801A99410090019105E0824229
:10ABB0009DD900230024009301940098019902B0CC
:10ABC0001CBC90469946A246F0BDA342A7D90022DC
:10ABD000002300920193B1E720224B46521AD34042
:10ABE0001A1C43468B401F1C174392E753462024F0
:10ABF0005646E41A3B1CB540E3401C1C2B1C234367
:10AC0000CDE7524620239B1A2A1C9A40271C131C6E
:10AC10005246D7401F43BBE720230022581A002387
:10AC2000009201930132C240019284E710B50029DD
:10AC300003D1FFF7B9FD203002E0081CFFF7B4FD97
:10AC400010BDC046C317C01858407047084B10B518
:10AC5000041C002B02D0002100E000BF054B186847
:10AC6000836A002B00D09847201C00F053FCC0469C
:10AC70000000000070BE00000E4B70B500251E1CC9
:10AC80000D4CE41AA410A54204D0AB00F358984729
:10AC90000135F8E700F040FC084B00251E1C084C6D
:10ACA000E41AA410A54204D0AB00F358984701352C
:10ACB000F8E770BD8C0400208C0400208C04002078
:10ACC00090040020002310B5934203D0CC5CC45400
:10ACD0000133F9E710BD031C8218934202D01970AA
:10ACE0000133FAE7704700000EB410B59DB002A919
:10ACF000029008610B48822488604861012040422C
:10AD00001FABC881084804CBA400006801938C8164
:10AD100000F074F80023029A13701DB010BC08BC38
:10AD200003B01847FFFFFF7F780000200023C25CBC
:10AD30000133002AFBD1581E70470000F0B58E6821
:10AD400085B0071C0C1C03920193B34245D390239A
:10AD50008A89DB001A423DD00325096923680198DE
:10AD60005B1A029363695D43EB0F5D19029B6D10E3
:10AD700001331B189D4200D21D1C381C53050FD5F2
:10AD8000291C00F01DFB061E13D0029A2169FFF753
:10AD900099FFA289184B134080221343A38111E02D
:10ADA0002A1C00F065FB061E0CD1381C216900F03E
:10ADB000C1FA0C23402201203B60A3894042134387
:10ADC000A38117E0029B2661F61826606561019E4B
:10ADD000ED1AA560019BB34200D2019E321C20688F
:10ADE000039900F092FA0020A3689B1BA3602368DC
:10ADF0009E19266005B0F0BD7FFBFFFFF0B59FB048
:10AE0000029005938B890E1C171C1B0610D50B692D
:10AE1000002B0DD1402100F0D3FA306030610028C2
:10AE200004D10C23029A01381360D0E040237361EF
:10AE3000002306AD6B6120336B761033AB763C1C80
:10AE40002378002B03D1E31B049312D003E0252BBE
:10AE5000F9D00134F4E7049B0298311C3A1CFFF747
:10AE60006DFF431C00D1ACE06A69049B94466344C7
:10AE70006B612378002B00D1A3E001220023524212
:10AE80006A6002A95432521801342B60EB60AB6047
:10AE90001370AB654F4F2178381C052200F02AFA59
:10AEA000002808D0C01B01278740381C2B680134BC
:10AEB00018432860EEE72B68DA0604D553222021D8
:10AEC00002A8121811701A0704D553222B2102A8C8
:10AED0001218117022782A2A01D0099B0EE0059AD7
:10AEE000111D12680591002A01DB099204E052420B
:10AEF000EA60022213432B60013409E02278303AE1
:10AF0000092A04D80A214B4301349B18F6E7099318
:10AF100023782E2B18D163782A2B09D1059B023474
:10AF20001A1D1B680592002B0DDA01235B420AE013
:10AF3000002301342278303A092A04D80A214B43ED
:10AF400001349B18F6E70793234F2178381C03221E
:10AF500000F0D0F9002807D0C01B40278740381CDC
:10AF60002B6801341843286021781C480622671C8E
:10AF7000297600F0BFF9002812D0194B002B06D11A
:10AF80000722059B073393430833059314E005AB71
:10AF900000930298291C321C124B00E000BF07E00E
:10AFA00005AB00930298291C321C0E4B00F08AF866
:10AFB0000390039B013304D06B69039A9B186B6168
:10AFC0003DE7B3890B985B0601D5012040421FB0D5
:10AFD000F0BDC04674BE00007ABE00007EBE000018
:10AFE000000000003DAD0000F7B5171C01930A6991
:10AFF0008B6800900C1C934200DA131C221C3B60EF
:10B0000043321278002A01D001333B6023689B064B
:10B0100002D53B6802333B60062523681D401ED0E5
:10B02000231C43331B785A1E9341226892061CD579
:10B030003020E1184031C870211C5A1C4531097874
:10B04000A21840320233D1700FE0221C0123009875
:10B0500001991932089EB047431C0ED00135E368B0
:10B060003A689B1A9D42F0DBDAE7221C00980199AE
:10B070004332089DA847431C02D10120404220E0F2
:10B0800006232068E1683A6803400025042B03D1B9
:10B090008D1AEB43DB171D40A3682269934201DD43
:10B0A0009B1AED180027AF420ADA221C01230098F0
:10B0B00001991A32089EB047431CDED00137F2E7EF
:10B0C0000020FEBDF0B58BB006920A1C43320793F8
:10B0D000059004920A7E0C1C109B6E2A00D1A8E0F9
:10B0E00011D8632A22D009D8002A00D1B2E0582A08
:10B0F00000D0C2E045310A707C4A4FE0642A1DD07E
:10B10000692A1BD0B9E0732A00D1A7E009D86F2AB9
:10B1100029D0702A00D0B0E0202209680A432260BA
:10B1200037E0752A1FD0782A33D0A6E00E1C1A68A3
:10B130004236111D196013683370A1E021681A6846
:10B14000080606D4490604D5111D19600023D55EF2
:10B1500002E0111D19601568002D3BDA2D23049AB9
:10B160006D42137036E021681A68080606D4490655
:10B1700004D51568111D1960ADB202E0111D1960EA
:10B1800015685A4B227E03930A276F2A1DD1082780
:10B190001BE0221C782145321170554A1968039230
:10B1A000081D226818600D68100602D4500600D5EC
:10B1B000ADB2D30702D520231A4322601027002DF9
:10B1C00003D1202322689A432260231C00224333A8
:10B1D0001A7002E00A27454B03936368A360002BB3
:10B1E00003DB0422216891432160002D02D1049EDB
:10B1F000002B0ED0049E281C391CFFF7D9F9039BA5
:10B20000013E5B5C281C3370391CFFF74BF9051EAF
:10B21000F1D1082F09D12368DB0706D563682269BD
:10B22000934202DC3023013E3370049B9B1B23615D
:10B230002BE009681A68080607D4490605D5111DD0
:10B2400019601368A28A1A8004E0111D196013683E
:10B2500062691A600023049E236116E01A68111DBA
:10B26000196016680021301C626800F043F800285D
:10B2700001D0801B6060636803E0261C4236327098
:10B28000012323610023049A1370079B0598009300
:10B29000211C069B09AAFFF7A7FE431C02D101202F
:10B2A000404221E0236905980699321C079DA84772
:10B2B000431CF4D023689B0705D4099BE06898429F
:10B2C00012DA181C10E00025E368099A9B1A9D42C7
:10B2D000F3DA221C0123059806991932079EB0471C
:10B2E000431CDCD00135EFE70BB0F0BD85BE00009C
:10B2F00096BE0000C9B28218904204D003788B42F7
:10B3000002D00130F8E70020704710B5814208D222
:10B310008B18984205D29B1A013A09D3995C815443
:10B32000FAE70023934203D0CC5CC4540133F9E71D
:10B3300010BD000030B500293ED004390B68002B49
:10B3400000DAC9181D4A1368141C002B02D14B6087
:10B35000116031E099420DD208680A189A4203D16F
:10B360001368C3180B6053684B60216024E08A4265
:10B3700003D8131C5A68002AF9D11D685C198C4245
:10B380000BD10968691858181960904214D11068D7
:10B390005268091819605A600EE08C4202D90C23D9
:10B3A000036009E008680C18944203D114685268DD
:10B3B000001908604A60596030BDC0467C0F00200B
:10B3C000032370B5CC1C9C430834051C0C2C01D203
:10B3D0000C2405E0002C03DA0C2300202B6042E053
:10B3E0008C42F9D3204A1368101C191C002913D071
:10B3F0000A68121B0DD40B2A02D90A608B181FE0B1
:10B400008B4202D15A6802601BE04A685A600B1CEA
:10B4100017E00B1C4968E9E7144E3368002B03D191
:10B42000281C00F04BF83060281C211C00F046F866
:10B43000031C421CD0D00322C61C964386420AD16C
:10B440001C60181C07210B301A1D8843821A0AD071
:10B450005142995007E0311A281C00F02FF8431C84
:10B46000BAD0331CECE770BD7C0F0020780F0020B1
:10B47000F8B5061C0C1C151C002904D1111CFFF783
:10B480009FFF041C18E0002A03D1FFF753FF2C1C78
:10B4900012E000F025F8A8420ED2301C291CFFF75C
:10B4A0008FFF071E07D0211C2A1CFFF70BFC301C46
:10B4B000211CFFF73FFF3C1C201CF8BD38B50023C2
:10B4C000064C051C081C236000F016F8431C03D131
:10B4D0002368002B00D02B6038BDC0469C0F002095
:10B4E0000B1F1A68101F002A04DA891804390B6828
:10B4F000D018043870470000044A1368002B03D0AA
:10B5000018181060181C7047014BF9E7800F0020D5
:10B51000A00F0020FEE7C046F8B5C046F8BC08BC46
:10B520009E467047F8B5C046F8BC08BC9E467047BA
:10B5300001B40248844601BC604700BF4D030020AF
:10B5400001B40248844601BC604700BFF9030020F3
:10B550005368617270204C53303133423744483065
:10B56000332023310000000005000000000000002F
:10B5700040420F0005010000000000000000000034
:10B5800001000100010000000100010000186C6CC6
:10B5900010CE3808600C0000000000007C307C7C7D
:10B5A000C6FE7CFE7C7C000070001C7C7C7C7E7C6B
:10B5B0007EFEFE7CC63C78C606C6C67C7E7C7E7C53
:10B5C0007EC6C6C6C6C6FE7C007C10000C00060007
:10B5D00060003800060000060C00000000000000BB
:10B5E000000000000000003018188C00000000006F
:10B5F00000186CFEFC6A2C1830186C18000000C093
:10B60000C638C6C6C606C6C0C6C61818387C38C6F0
:10B61000C6C6C6C6C60606C6C618306606EECEC67E
:10B62000C6C6C6C618C6C6C6C6C6C00C06603800A2
:10B630000C00060060000C00061830060C0000002C
:10B640000000000018000000000000181830D600AC
:10B6500000000000001848FE162E2C18183038186C
:10B6600000000060C63060C0C6060660C6C6181876
:10B670001C7C70C6F6C6C606C6060606C618303658
:10B6800006FEDEC6C6C6C60618C6C6C66CC6600CB2
:10B690000C606C00043C3E3C7C3C3C3C3E00006644
:10B6A0000C6E3E3C3E3C363C186666C666667E18AE
:10B6B00018306200000000000018006C7C10DC00F4
:10B6C0001830FE7E1C7E0030C6303070FE7E7E302C
:10B6D0007CFC00000E00E070F6FE7E06C61E1EF624
:10B6E000FE18301E06D6F6C67EC67E7C18C6C6D6A6
:10B6F00038FC300C1860C6000060660666660C6692
:10B70000661830360CD6666666666E067C6666C659
:10B710003C66300C0060000000000000000000FEED
:10B72000D0E866001830387E1C7E1C18C63018C061
:10B73000C0C0C618C6C018181C7C703076C6C606B5
:10B74000C60606C6C618303606C6E6C606B6C6C063
:10B7500018C6C6FE6CC0180C30600000007C66067F
:10B76000667E0C7C6618301E0CD666663E56063C1D
:10B77000186666D6187C1818183000000000000003
:10B78000001800FE7EAC660030186C1818001C0C07
:10B79000C6300CC6C0C6C60CC6C61818387C3800E1
:10B7A00006C6C6C6C60606C6C618366606C6C6C6D7
:10B7B0000666C6C618C66CEEC6C00C0C606000FEFD
:10B7C0000066660666060C60661836360CC6666647
:10B7D0000626066018663CD63C600C18183000003F
:10B7E000000000000018006C10E6DC00600C00187F
:10B7F0000C001C067C78FE7CC07C7C067C7C000CEB
:10B8000070001C307CC67E7C7EFE06FCC63C1CC6DE
:10B81000FEC6C67C06DCC67C187C38C6C67EFE7CAE
:10B82000C07C00FE007C3E3C7C3C0C3E66701C668E
:10B8300038C6663C065C063E707C18FC663E7E3070
:10B8400018180000000000000000000000000000C8
:10B8500000000000000000000000000000000000E8
:10B8600000000000000000000000000000000000D8
:10B8700000000000000000000000000000000000C8
:10B8800000000000000000000000000000000000B8
:10B8900000000000000000000000000000000000A8
:10B8A0000000000000000000000000008CB5000057
:10B8B0002003016408080200010000004E29000076
:10B8C0006E29000096290000B6290000EE2900002C
:10B8D000EE290000DE2900009A3000000830000048
:10B8E0009A3000009A3000001A3000003230000018
:10B8F0004A30000072300000F8310000E4300000EF
:10B90000F8310000F83100001C3100004E31000019
:10B9100094310000C6310000A03200004232000025
:10B92000483200003C320000A0320000A03200008B
:10B930004E3200005832000062320000A032000097
:10B940006E320000BE350000343400009C3400002C
:10B95000E834000034350000BE35000066350000D4
:10B9600070350000F83700001E360000A8360000D1
:10B97000A836000036370000F8370000F83700001E
:10B9800084370000FC370000FC370000323600002E
:10B99000403600004E3600005C360000FC370000E8
:10B9A000FC370000FC370000FC3700006A3600005E
:10B9B000FC37000000380000BC360000C236000032
:10B9C000D23600000038000000380000E2360000E7
:10B9D0000038000000380000003800000038000087
:10B9E000F4360000423800004E3800005E38000097
:10B9F0006E380000783800005039000042390000ED
:10BA0000263900001839000034390000623900007E
:10BA100008091108C64100001C420000A2420000B3
:10BA2000F042000046430000944300001C44000024
:10BA300064440000FC44000003000000000000001B
:10BA40001E000000010101010000030203000000CC
:10BA50000002030000000000010000000BEE42E7BE
:10BA60005FDF21DAF9D55ED598D827DE76E47EEC63
:10BA7000EBF177F6F6FA22FE3C019D0403086A0C0E
:10BA8000EF113918F41E4B241B285E2858259F1FE0
:10BA90001C19E012A10DFC086105200272FF7CFC5C
:10BAA000AEF84DF4CA115D0CD6073304E8000AFE67
:10BAB0007FFA89F6FFF100EB67E4FCDDC1D726D5FC
:10BAC000FCD517DA3CDFEFE585EC79F236F713FBAE
:10BAD0008AFE9F0136056509650E3314581AFE204B
:10BAE000CA255B289027B723CA1D7A172025642012
:10BAF0004465672000000000436F6E6E656374004C
:10BB00005369373278782D4558500000507265736C
:10BB1000732052657365740044656D6F204D656ECA
:10BB20007500000050423120746F205363726F6CB7
:10BB30006C00000050423020746F2053656C6563C8
:10BB4000740000002D3E000020204558502057680A
:10BB500065656C0020204558502052657620436E64
:10BB60007400000020205053204932432044617467
:10BB70006100000020205053204932432054656D5D
:10BB800070000000202050532053772F4C617463C5
:10BB9000680000002020505320416E616C6F6700E8
:10BBA000202050532050574D0000000020205053BB
:10BBB0002053454E5400000055323A202533642E60
:10BBC0002531646D5400000055313A202533642E30
:10BBD0002531646D54000000416E676C653A202584
:10BBE000336C640054414D50455200005265766FED
:10BBF0006C7574696F6E0000436F756E743A202522
:10BC000064000000517561643A2531640000000051
:10BC1000505320426F617264000000005369373254
:10BC20003130204932430000436F6E6E65637420EB
:10BC3000505300003230306D54205363616C650006
:10BC400032306D54205363616C6500004669656C49
:10BC50006420537472656E67746800002025642E3A
:10BC60002531646D5400000050423120746F206310
:10BC700068616E67650000006D54207363616C65D8
:10BC80000000000054656D70657261747572650026
:10BC900054656D703A2025336C642E253031644331
:10BCA000000000004F555450555420537461747572
:10BCB0007300000053693732303120537769746361
:10BCC00068000000536937323032204C6174636879
:10BCD0000000000048494748000000004C4F570052
:10BCE00053693732313120416E616C6F670000005B
:10BCF0002533642E25303164206D5400566F7574E1
:10BD00002F56646420282563290000002532642E04
:10BD10002530316400000000536937323132205041
:10BD2000574D0000447574792D4379636C650000AC
:10BD300050574D282563292533642E253031640062
:10BD40005369373231332053454E54004E69626295
:10BD50006C6520446174610025346400526576315D
:10BD6000203A204E4F540000434F4D504154494219
:10BD70004C4500005245504C41434500424154540B
:10BD8000455259005662617420746F6F204C6F7772
:10BD9000200000002055736520555342206F72200B
:10BDA000000000006E65772062617474657279002E
:10BDB000746F2063616C69627261746500000000D9
:10BDC000576865656C20506F736974696F6E000009
:10BDD00043616C6962726174696F6E005475726E52
:10BDE00020776865656C20746F0000005468656E8C
:10BDF00020707573682050423100000000060D135A
:10BE0000191F24292E3236393B3D3E3E00000100E9
:10BE1000000001000100000000010100000001001D
:10BE2000010000000001010000000101010000000C
:10BE3000EAA10000F0A10000F6A10000FCA10000B2
:10BE400002A2000008A200000EA2000014A200003E
:10BE50001AA2000000A00040030703060100000032
:10BE600000000000486B01000000000043000000DB
:10BE700018000020232D302B2000686C4C006566D4
:10BE8000674546470030313233343536373839412B
:10BE90004243444546003031323334353637383941
:0CBEA00061626364656600000000000041
:08BEAC004842FF7F0100000085
:10BEB40000366E0100800000410400000000000014
:10BEC400EC0400200010000000000000000000004E
:10BED400000000000000000000000000000000005E
:10BEE40000000000000000006CBE00000000000024
:10BEF400000000000000000000000000000000003E
:10BF0400000000000000000000000000000000002D
:10BF1400000000000000000000000000000000001D
:10BF240000000000000000001800002080B582B06E
:10BF340000AF78603960FEE780B584B000AF786008
:10BF4400184BFB6002E0FB68013BFB60164BDB69AE
:10BF54000122134002D0FB68002BF4D1FB68002BB4
:10BF640001D1FD2319E0104B7A681A610E4B0122AE
:10BF7400DA600D4BDB69BB60BB68062213400BD053
:10BF8400BB680422134001D0FF2306E0BB680222F1
:10BF9400134001D0FE2300E000235BB2181CBD4611
:10BFA40004B080BD8096980000000C4080B58AB033
:10BFB40000AFF860B960FB1D1A701F23FB18002244
:10BFC4001A700123BB61BB68002B00D193E0FB1DF9
:10BFD4001B78002B43D100233B623BE04A4AFB68B9
:10BFE400191DF9601B6893613B6A01333B62BB69AD
:10BFF400012B03D1444B0822DA6014E0BB69022B05
:10C0040011D1C046404BDB6908221340FAD03E4AA6
:10C01400FB68191DF9601B6893613B6A01333B623D
:10C02400394B0822DA60394B7B6202E07B6A013BC0
:10C034007B62354BDB690122134002D07B6A002B03
:10C04400F4D17B6A002B05D11F23FB18FD221A7043
:10C05400C04650E03A6ABB689A42BFD34BE0EFF364
:10C0640010833B613B697B6172B600233B6225E030
:10C0740008E0254BDB6919221340102B02D1224B17
:10C084001022DA60204BDB6908221340F1D01E4AEB
:10C09400FB681B689361BB69012B06D0BB69022B4B
:10C0A40006D13B6A0122134002D0174B1022DA60FA
:10C0B400FB680433FB603B6A01333B623A6ABB684A
:10C0C4009A42D5D37B69002B00D162B60F4B7B62B9
:10C0D40002E07B6A013B7B620B4BDB69012213406C
:10C0E40002D07B6A002BF4D17B6A002B03D11F237F
:10C0F400FB18FD221A701F23FB181B785BB2181C57
:10C10400BD460AB080BDC04600000C408096980031
:10C1140090B58BB000AFF860B9607A601A1CFB1C54
:10C124001A701B23FB1800221A70334B324A926890
:10C1340001210A439A607B689B087B6100237B6230
:10C14400BB68FB6146E07B6A9B00FA68D3181B223C
:10C15400BC18181CFFF7F0FE031C23701B23FB18EC
:10C164001B785BB2002B03D01B23FB181B783EE02B
:10C174007B6A9B00FA68D3189B059B0D8022D20032
:10C18400D31A9B083B627A697B6AD21A3B6A9A4249
:10C1940003D27A697B6AD31A3B621B23FC18F969C0
:10C1A4003A6AFB1C1B78081C111C1A1CFFF7FEFEC4
:10C1B400031C23701B23FB181B785BB2002B00D0DD
:10C1C4000CE07A6A3B6AD3187B623B6A9B00FA698B
:10C1D400D318FB617A6A7B699A42B4D3064B064A48
:10C1E400926801218A439A601B23FB181B785BB277
:10C1F400181CBD460BB090BD00000C4080B584B047
:10C2040000AF7860264BFB60264B264A92680121DA
:10C214000A439A60234B7A681A61224B0122DA603E
:10C22400204BDB690422134007D01E4B1D4A926841
:10C2340001218A439A60FF232DE01A4BDB69022215
:10C24400134007D0174B174A926801218A439A601A
:10C25400FE2320E0134B0222DA6002E0FB68013B7C
:10C26400FB60104BDB690122134002D0FB68002BFA
:10C27400F4D1FB68002B07D10A4B0A4A92680121CA
:10C284008A439A60FD2306E0064B064A9268012120
:10C294008A439A6000235BB2181CBD4604B080BD7B
:10C2A4008096980000000C4080B584B000AFF86020
:10C2B400B9607A60F968BA687B68081C111C1A1C9A
:10C2C4000023FFF725FF031C181CBD4604B080BDE6
:10C2D40080B584B000AFF860B9607A60F968BA6874
:10C2E4007B68081C111C1A1C0123FFF711FF031C97
:10C2F400181CBD4604B080BD80B500AF0D4B0D4A7F
:10C30400926801210A439A600A4B0B4A5A65094B09
:10C3140080225200DA60C046064BDB6901221340DA
:10C32400FAD1044B00225A6500235BB2181CBD46A7
:10C3340080BDC04600000C401A630000BD00000030
:08C3440095000000000000005C
:040000030000016D8B
:00000001FF
